:100000000C94071B0C942E1B0C942E1B0C944F2C41
:100010000C942E1B0C942E1B0C942E1B0C942E1B3C
:100020000C942E1B0C942E1B0C942E1B0C94981DC0
:100030000C942E1B0C942E1B0C942E1B0C942E1B1C
:100040000C942E1B0C942E1B0C942E1B0C942E1B0C
:100050000C942E1B0C942E1B0C942E1B0C942E1BFC
:100060000C942E1B0C942E1B0000E0FF10841F002C
:10007000228A10806636FF070F044A616E7561722E
:100080000046656272756172004DC3A4727A0041C8
:100090007072696C004D6169004A756E69004A753D
:1000A0006C69004175677573740053657074656D94
:1000B000626572004F6B746F626572004E6F766599
:1000C0006D6265720044657A656D626572004DC34C
:1000D000BC6C6C6B616C656E6465720000001FF82F
:1000E00000F8E0071F00E0FF20253032643A253099
:1000F00032643A253032642000536F6E6E7461674B
:10010000004D6F6E746167004469656E737461675A
:10011000004D697474776F636800446F6E6E65722A
:1001200073746167004672656974616700536F6E2E
:100130006E6162656E64002025642E2025532025A3
:10014000642530326420002025532000E0FF0000A9
:100150000000FFFFFFFFFFFF0000FFFFFFFF4B65F9
:10016000696E20416266616C6C00427261756E65F9
:1001700020546F6E6E6500426C61756520546F6E21
:100180006E6500477261756520546F6E6E6500473D
:10019000656C626520546F6E6E6500686575746588
:1001A000006D6F7267656E00C3BC6265726D6F72C1
:1001B00067656E00AC2020001A2092011E202620C8
:1001C00020202120C6023020600139205201200069
:1001D0007D0120002000182019201C201D20222035
:1001E00013201420DC02222161013A205301200057
:1001F0007E0178010000E5F07801000002000203B2
:10020000301004000010000011070012000013005D
:1002100000070100FFC800109016112702FF3200EE
:10022000120D00FF3200130012290A00FF320030C5
:100230000000310007320707350000360F0037078E
:10024000073807003900003C00003D000FFE0000A9
:10025000600027610300901000920000073301FC4A
:100260001320E00054C5081152100055555555553E
:100270002255657C88788608859688877886B87741
:10028000151055515656620650A066665261956526
:100290002520551550C455E1171C15014024C5C132
:1002A000151B7500555550815215585211510511A5
:1002B0005299697777778C77770011888888588882
:1002C0008878675555555A555500116666665666C5
:1002D00066666600000000000000000000000000EC
:1002E000000000000000000000000000000000000E
:1002F00000000000000000000000000000000000FE
:1003000000000000000000000000000000000000ED
:1003100000000000000000000000000000000000DD
:1003200000000000000000000000000000000000CD
:1003300000000000000000000000000000000000BD
:100340000000000000000000001F00000000F80096
:100350000000000000000000000000000000003667
:10036000000000000000000000000000000000008D
:10037000000000000000000000000000000000007D
:10038000E00E0380E81B01E00000000380380E034C
:10039000639DDB0000E80E00700700E80D800000A0
:1003A00007003803806C0700000000000000000018
:1003B000000000000000000000000000000000003D
:1003C000000000000000000000000000000000002D
:1003D000000000000000000000000000000000001D
:1003E000000000000000000000000000000000000D
:1003F00000000000000000000000000000000000FD
:1004000000000000000000000000000000000000EC
:1004100000000000000000000000000000000000DC
:1004200000000000000000000000000000000000CC
:1004300000000000000000000000000000000000BC
:100440000000000001C00000000E000000000000DD
:100450000000000000000000000006C000000000D6
:1004600000000000000000000000FF80000000000D
:1004700000000000000000000000000C0180F817E0
:1004800003603C00000000300603E06C337F600036
:100490001700C00C01F01701B0000000600600F862
:1004A0000D80C000000000000000000F00000000F0
:1004B000000000000000000000000000000000003C
:1004C000000000000000000000000000001000001C
:1004D000000000000000000000000000000000001C
:1004E000000000000000000000000000000000000C
:1004F00000000000000000000000000000000000FC
:1005000000000000000000000000000000000000EB
:1005100000000000000000000000000000000000DB
:1005200000000000000000000000000000000000CB
:1005300000000000000000000000000000000000BB
:1005400000000000000000000000000000000000AB
:10055000000000000000000000000000000000009B
:1005600000000000001FF00000000000000000007C
:1005700000000000000000000000000000078000F4
:10058000000000000000000000000000000000006B
:100590000000000000000400000000000000000057
:1005A00000000000000001E000000000000000006A
:1005B000000000000000000000000000000000003B
:1005C000000000000003330D8F8F0E03E0C7E10031
:1005D00000003BF030FC7E071F87CFF3F1F00000F6
:1005E000000000FC07F80E0FF03F8FF0FF9FE1FCCA
:1005F000606603307300F1E7061F87F83F0FF87F4E
:100600003FF606C06E38FE1F03BFDF9E3C00380079
:100610006000003001F001806660300000000000E2
:10062000000000180000000000000007B780000074
:10063000F8000F00000018061DF3801FC00FFF8197
:10064000FE00331B3600000000EBEC61F000000000
:100650007CC0E000C3E0039CC7CD8FC7C00000078B
:10066000E001F003FF7001FE0073E0071C38E3E3D4
:100670000000700E01C0380700F03FFC3F8FF9FF0B
:100680003FE7FCCCC63FC3830FC0FC0FC0FC0FC0CC
:10069000007FD81981981981B03B003E0701C1C184
:1006A000D0D83C000000381C0E0D9CEED8F83A075C
:1006B00001C0703A0D800000700E0381B038600DEB
:1006C000806663F3FBF1C0FE18FCF80000077E0EA5
:1006D0003FDFE0E7F1FDFEFF7F00000000003FC1CB
:1006E000FF83E1FF0FF9FF1FF3FC7FCC0CC0661CFA
:1006F000601E3CF0C7F8FF8FF1FF9FF7FEC0DC1DC6
:10070000CF9DC770E7FBFBC78003000C000006000D
:100710003E00300CCC06000000000000000003008A
:1007200000000000000000F6F000FE3F7C03E00047
:10073000000300C7FEE007FC03FFFFBFFFF6636690
:10074000C00000001711DC1C000007C71C3800188F
:10075000FE007398FDB79EF8000003CF0036187FA7
:10076000EC007FC01E7C01E30F387CE0001F03E03B
:100770007C0F81F03E07FF8FF9FF3FE7FCFF999860
:10078000C7FC7863FC3FC3FC3FC3FC001FF303308E
:10079000330330370E600FE060307C2E1B07800083
:1007A00000030303E1B19BFB1E05C060301F05C1C0
:1007B000B00000060180F836060C01B00CCC7E7F3C
:1007C00066701DC339CE0C0000FCE7C73B9C3CE0C3
:1007D0007B81DCEE700001801807B87CF87C30E388
:1007E000CF30F300601E7981980CC70C03C79E19A7
:1007F000E79873CF30739E0C181B83B9F39DC738ED
:100800000E6719F8000001800000C0060006000114
:1008100080C0000000000000000060000000000038
:1008200000001CCE0018CF6D80700000006018061C
:10083000DC00E780F781B076F684484800000000CD
:10084000023B80000000D801CE00031DC826631FB4
:1008500080C0CF00000060600443039C000FB00024
:10086000CD800CE06703980003E07C0F81F03E0729
:10087000C0F803CF300600C018033318C3CF0CF301
:10088000CF3CF3CF3CF3C0079E60660660660673FC
:100890008FF1DC00000000000000000000000000FC
:1008A00000000007E0000000000000000C00400015
:1008B0000000000001800001999FCD0CCE03B867B5
:1008C0003BE180001F9CF8C303879C0E00730D86DC
:1008D00030C0F7FBC0E31DFF8D860C70E60E600C88
:1008E000038730330199C18078F3E338730670E6EB
:1008F0000671C1830338E3BE63F8E701CCE33F0030
:10090000003F3F87E3F8F9F1FCDE3333D9FBE7F032
:10091000FC7F0FE7CF9F61B8FCE7E3E0CFE318C0AF
:100920000319C1B00E0000000C1FE0DF001C701C9A
:1009300070360EDED98D9B000000000045D0F80314
:10094000FF9B7F39C067E33BFEFC63C033CFE0070A
:10095000F81BE600D860F1818DF60019B001980D02
:10096000C03700C06C0D81B03606C0D83B0070E6C1
:1009700000C018030066631839F19C39C39C39C361
:100980009C3B98E3CC0CC0CC0CC0CE71FF3387E30A
:10099000F1F8FC7E3F1FF87E3E1F0F87C66630FCD5
:1009A0007F0FC3F0FC3F0FC181FCC330CC330D83FC
:1009B0003F98303003F9E1FB807F00E7003000030F
:1009C000E19B00E1F1F3F9FC1C73B0C6187EFF7ED9
:1009D00000E7FFF3B8C38E00C1CC0180700606604B
:1009E0003378300FBE6C670E61CE1CC3CF80306091
:1009F000671C77DC3E0FC0719C6E70000FE7F9FC3E
:100A0000FF3FBE7F9FE666F33FFCFF3FCFF3FCFB5B
:100A1000FBEC331BBEEEEE39FC631800637F360738
:100A2000E000000FF3FC1FE003E0730606C39BDB4E
:100A300031B363E000000008BA3F9CFFFB6FE3F0B6
:100A40000DFE703F9F8C7C06CDFC7EFF034CC01FCB
:100A50007FBDF031BEC0033EFC3701B83EC0181D5B
:100A6000C3B8770EE1DC3B87600E00C0180300605E
:100A70000CCC63073633873873873873877F9CF9CC
:100A8000819819819818FC30E671FCFE7F3F9FCF5A
:100A9000E7FF9FCFE7F3F9FCCCC63FCFF3FCFF3F66
:100AA000CFF3FC007F1866198661B8E7FB8E06005D
:100AB0003F3F1EE00FC01CE03FC0006C30601C3E9A
:100AC000767FBFC38FE738003F0003F03CFEF67728
:100AD0001FF1801819FF3F8C00FFCC067F0601F73D
:100AE000CDCCC0CFF9819FF8FE060C0C670EDB83DE
:100AF00080F01C338DCE0001DCE73B9CE7730E7366
:100B0000DCCCFC677B9EE739CE739D7731867777A7
:100B1000DCF9C7039C639F6C6606C0FC000001FE05
:100B20000C03F8003F8E60FFD8E37B0000007C00E0
:100B30000000011747739CF76C1C3C003BDF87717A
:100B4000E19FC0901F8FC0604988000FF7FE0633F9
:100B5000D80067DF86E03607F80003B8770EE1DCDF
:100B60003B8771CFF9801FF3FE7FCFF9998CFC662C
:100B7000E66066066066066067E33B303303303349
:100B8000030F060CCC3B9DCEE773B9DCEF73B9DCE9
:100B9000EE773B9998C739EE739CE739CE73BFCE99
:100BA000F30CC330CC371CE771C0C006C3F01DE3A3
:100BB000FB030C07F8001D860C0F01CCCE773871B3
:100BC000FEFF000783FC1E0F1F8EDC73FF30030344
:100BD0003FE7F18F9FF980CFF0C036D99D9819FE7D
:100BE0003033FE0FE0C1818EE0FBF0701E038631D2
:100BF0008000000F9CE6039CFE61CE71999F0CC79C
:100C0000338CE739CE738F8630CEE6FB1F1DC0E7ED
:100C10008C7BFD8DFCD80E00000006018007FBE3F5
:100C2000FB8C1FFB1C6F6000000F800000000000A9
:100C3000F83B9FED87078037C3F0C6FF03BC120265
:100C400003F00C09F10000300000C61B300001F871
:100C500039C1FE067060E39C738E71CE39C739FFCF
:100C60003003FE7FCFF9FF33318C0CCECC0CC0CCDF
:100C70000CC0CC0C786E66066066066061E0C199B7
:100C8000C1F0F87C3E1F0F87FE603F9FCFE7F33334
:100C900018E738CE739CE739CE77F9FE619866196C
:100CA00086771CE7701801FC1E077E77E0618018CC
:100CB00003C3B0C183C01B9806C31C39CFE000FC3E
:100CC0007F8FC1C363FBFE61E70060E600C039F3BC
:100CD000033019CE1806FB31B30330060667803C9B
:100CE000183031DC1F7C1F0180E0C730000007F3A3
:100CF0000CC0619FCC30CC3333F198C66198661933
:100D00008661FCC618F8FFE1C3B838F18F4FB1BC5B
:100D10001B01C0000000C03000DF7C0F71C70367FB
:100D20000DEC000001FFFFFFF800001FC761FDB1DF
:100D3000C06006D8181DC300638366C07E019FA6ED
:100D4000600006000018C36600003F07383FC1CEB0
:100D50001C1FF3FE7FCFF9FF3FEFF00700600C018F
:100D600080300666318398D9819819819819819FBE
:100D70008F9CC0CC0CC0CC0C1818733CFE7F3F9FDE
:100D8000CFE7F3FFCC07F3F9FCFE6663186619861C
:100D900061986619860036CC330CC330CEE30CEE76
:100DA00003003F9AC0ECCC7C0C30030078773830DD
:100DB000F0E37FB8D86386181C0007E007E0306CCA
:100DC0007F7FCC0CE1CC1CC01807066066C330E303
:100DD00000DF663E70E600EDCC78E183070E1F036E
:100DE000EF87F0303818E6000000FE73980E7301AC
:100DF000873986667E3318CC339CE739CC0F98C789
:100E00001F1F7C7C7E0E0E31C006338360380000CD
:100E1000001806003B6DB86E38E06DC1BD80000063
:100E20003FFFFFFF000000F8EE7036700C00DFE7B8
:100E300003FBFC0F7067980FC033F4CC0000C000B8
:100E400003986C000007E1CF0E3833C783FE7FCFD5
:100E5000F9FF3FE7FDFE00E1CC0180300600CCC683
:100E600030731F3873873873873877F9E39C39C339
:100E70009C39C38303FE639FCFE7F3F9FCFE7B013C
:100E800080C06030180CCC639CC339CE739CE739AA
:100E9000C307F98E6398E639F8739F800007E3F87B
:100EA0003999CF81CE0060000EE7061C1CEFF73B9E
:100EB000DC70E77780003C00F0000DDFDC1D839ED6
:100EC0007987980300F3CC0CDDE61C6019CCC3CF06
:100ED0003CC01FF9879E7060F3C3E07DF0EE06070B
:100EE000031CC000001DCE73B9CE7730E730CCCCE8
:100EF000E6631986739CE77987731DE3E3EF8F87B9
:100F0000C380C63000C67B6C070000000300C0072A
:100F10006DB79CE7BC0DB837B000000000000000C2
:100F200000007739CF76DC01801BDDFBFF8C19FEDA
:100F3000060600FC0003030000000000770D80009F
:100F400001F83B61CF0ED9E0E0FC1F83F07E0FC1BA
:100F5000F8C01E7980300600C01998C61E61E79E51
:100F600079E79E79E79EE73CF3CF3CF3CF3CF06016
:100F70007F8DF3B9DCEE773B9DCEF73B9DCEE773DB
:100F8000B9998C73986739CE739CE73860F73BCE7C
:100F9000F3BCEF1F0E71F00C00FC7F0E3F3FF839E1
:100FA000C000180DCFC0C7FBFC0CFF3F8C1FEFE14A
:100FB0008601801800C1FFFB83BFF1FF3FE3FE60A5
:100FC0000FF9819BFCC1CFF3399878FF1801FE30EF
:100FD00073FE0C1FF838071C38E0C1FF639800004F
:100FE00003FDFE7F3FCFE61FE619999CCC6330CF0F
:100FF000F3FCFF30FE7BFC383DE3B8F87F18C600F9
:1010000018C7EDB0C1B18C6060FF01CFBEFF9C7FFF
:10101000FFBFFEF60000000000000000000FE73FE9
:10102000FEDBF830037FBFE821830F8073801F80D1
:101030000039C0001FE0000FE1B000003F0E7E73DA
:10104000C19FB81C1F83F07E0FC1F83E1FF1FF3F08
:10105000E7FCFF9FF33318FF8C3C7F87F87F87F80E
:101060007F8007FC7FE7FE7FE7FE0C0C01BE7FBFA1
:10107000DFEFF7FBFDFFE7F3F9FCFE7F33318FF382
:101080000CFF3FCFF3FCFF001FE7F9FE7F9FE3E17A
:10109000FE3E01801F87C1C3C3F60738000301B1BC
:1010A000F818FF3F018FC3E181F8F830C00000005D
:1010B000183BFE7077FC1FC7F87FCC00FC30333F35
:1010C000181DFE6733070FC3001FE60F3F8181FE27
:1010D0000700E38E1E183FEC730000003FBF87C37C
:1010E000F8F8C1ECC33331D98C6618FC7F0FE60FDA
:1010F0008F3F87071CE38E0FE318C003F87DF63897
:1011000036318C0C1FE039F7CFE007FFFFFFFFC03F
:10111000000000000000000000F803FF9F7F0600B1
:1011200067E67C003060F007E000000003F0000399
:10113000FC0001FC3600000001C18E7C70663B8320
:10114000F07E0FC1F83F07C3FE1FC7FCFF9FF3FEF1
:1011500066631FE18387E07E07E07E07E001FF070B
:10116000F87F87F87F8181803387F3F9FCFE7F3F2A
:10117000BEF87C3E1F0F87C66630FC618FC3F0FC53
:101180003F0FC003F87F1FC7F1FC383F838000008A
:10119000002000000000E700002000000000000028
:1011A0000000000000000008000000000380700044
:1011B000000000000000000000000000000000002F
:1011C00000000000000C0000000000000000000013
:1011D000000001806000000000000000000073803B
:1011E00000E000000000000C000C00000000000007
:1011F0000003C00073380000000047024000018077
:10120000600000000000000000000000000000007E
:1012100000000000000000000000000CC000000002
:101220000CEE00000000000000000000000030068E
:10123000C0E000000000000000E700000000000027
:101240000000000000E000000000000000000000BE
:10125000000000000000000000100000000000007E
:101260000000000000000000000000000007000077
:10127000000000000000000000000000000000204E
:1012800000000000000F0600F00000000000000059
:10129000000FC0000C000000000000000000000073
:1012A00000000300000000007E3E0000000000007F
:1012B000000000000000000000000000000000002E
:1012C00000000000000000000000000000003C3CA6
:1012D00000FF800000000000000FF0001C00000074
:1012E00000000180018000000000000000F0000FFD
:1012F0006F000000001BE0D80000300C0000000070
:1013000000000000000000000000000000000000DD
:101310000000000000000198000000019FC00000D4
:101320000000000000000000000600D81C000000C3
:10133000000000001FE000000000000000000000AE
:101340001C00000000000000000000000000000081
:10135000000000000000000000000000000000008D
:10136000000000000000000000E00000000000009D
:10137000000000000000000000000000000000006D
:1013800003C0C03C000000000000000001F80001A4
:10139000800000000000000000000000000060006D
:1013A00000000007FF8000000000000000000000B7
:1013B000000000000000000000000000000000002D
:1013C0000000000000000000000787801FF0000000
:1013D0000000000000FC000380000000000030005E
:1013E00030000000000000001E0001EDE0000000E1
:1013F00003781B00000601800000000000000000D0
:1014000000000000000000000000000000000000DC
:101410000000330000000031F00000000000000078
:101420000000000000C00007800000000000000174
:10143000F80000000000000000000007800000002D
:10144000000000000000000000000000000000009C
:10145000000000000000000000000000000000008C
:10146000000000003C000000000000000000000040
:101470000000000000000000000000007818078055
:10148000000000000000000000000000000000005C
:101490000000000000000000000000000000003F0D
:1014A000C00000000000000000000000000000007C
:1014B000000000000000000000000000000000002C
:1014C000000000000000000000000000000000001C
:1014D000000000000000000000000000000000000C
:1014E0000000000000000000007FC01F000000009E
:1014F00000000000000000000003E00FFC000000FE
:1015000000000000000000000001F00000000000EA
:1015100000000000000000000000000000000000CB
:1015200000000000000000000000000000000000BB
:1015300000000000000000000000000000000000AB
:10154000000000000000000000000000000000009B
:10155000000000000000000000000000000000008B
:10156000000000000000000000000000000000007B
:10157000000000000000000000000000F01820E063
:1015800006070A0C0C110F050707080C06070606CC
:101590000C0C0C0C0C0C0C0C0C0C07070C0C0C0D94
:1015A000140F0F0F0F0E0D100E050C0F0D110E1056
:1015B0000E100F0E0D0E0D150E0E0C0706070C0C5F
:1015C000070C0D0C0D0C080D0D05050C05130D0D6C
:1015D0000D0D080C070D0D0F0C0C0B0806080C0B5D
:1015E0000C07060C0B150C0C07150E0715070C073E
:1015F0000706060B0B070C1507150C0714070B0E37
:1016000006070C0C0C0C060C070F080C0C070F0C33
:10161000080C0707070C0C060707080C1212120D1E
:101620000F0F0F0F0F0F150F0E0E0E0E05050606EE
:101630000F0E10101010100C100E0E0E0E0E0E0DC0
:101640000C0C0C0C0C0C130C0C0C0C0C05050606ED
:101650000D0D0D0D0D0D0D0C0D0D0D0D0D0C0D0CBD
:10166000000000000000000000000000000000007A
:10167000000000000000000000000000000000006A
:10168000000000000000000000000000000000005A
:10169000000000000000000000000000000000004A
:1016A000000000000000000000000000000000003A
:1016B000000000000000000000000000000000002A
:1016C000000000000000000000000000000000001A
:1016D000000000000000000000000000000000000A
:1016E00000000000000000000000000000000000FA
:1016F0000000000000000000000077000000000073
:101700007700000000000000000000000000000062
:1017100000000000000000000000000000000000C9
:1017200000000000000000000000000000000000B9
:1017300000000000000000000000000000000000A9
:10174000000000070003801F007F00000000000071
:101750000000001C001C01F0000387F8000001FCE1
:1017600001C000E001F003F80000000000003800B4
:101770007003E000001C00000000000000000000FA
:101780000000000000000000000000000000000059
:101790000000000000000000000000000000000049
:1017A0000000000000000000000000000000000039
:1017B0000000000000000000000000000000000029
:1017C0000000000000000000000000000000000019
:1017D0000000000000000000000000000000000009
:1017E00000000000000000000000000000000000F9
:1017F00000000000000000000000000000000000E9
:1018000000000000000000000000000000000000D8
:1018100000000000000000000000000000000000C8
:1018200000000000000000000000000000000000B8
:1018300000000000000000000000000000000000A8
:101840000000003E00000000003E0000000000001C
:101850000000000000000000000000000000000088
:1018600031800000000000000000000000000000C7
:101870000000000000FFF000000000000000000079
:1018800000000000000000000000000003800700CE
:101890001F007F00C6007800000000000E00380125
:1018A000F00C61CEFA300001FC00E001C001F00351
:1018B000F80318000000001C00E003E018C0380026
:1018C0000000000000000000000000000000000018
:1018D0000000000000000000000000000000000008
:1018E00000000000000000000000000000000000F8
:1018F00000000000000000000000000000000000E8
:1019000000000000000000000000000000000000D7
:1019100000000000000000000000000000000000C7
:1019200000000000000000000000000000000000B7
:1019300000000000000000000000000000000000A7
:101940000000000000000000000000000000000097
:101950000000000000000000000000000000000087
:101960000000000000000000000000000000000077
:101970000000000000000000000000000000000067
:101980000000000000000000000000003E00000019
:1019900000003E0000000000000000000000000009
:1019A0000000000000000000003180000000000086
:1019B0000000000000000000000000000000FFF038
:1019C0000000000000000000000000000000000017
:1019D0000000000000038007003B805F00C6007825
:1019E00000000000000E003803B80C61CEDE3000AD
:1019F000017C00E001C003B802F8031800000000F9
:101A00001C00E0077018C038000000000000000053
:101A100000000003C0000000000000000000000003
:101A200000000000000000000000000000000000B6
:101A300000000000000000000000000000000000A6
:101A4000C0000000000000000000000000000000D6
:101A50000000000000000000000000000000000086
:101A60000000000000000000000000000000000076
:101A70000000000000000000000000000000000066
:101A80000000000000000000000000000000000056
:101A90000000000000000000000000000000000046
:101AA0000000000000000000000000000000000036
:101AB0000000000000000000000000000000000026
:101AC0000000000000000000000000000000000016
:101AD0000000000000000000000000000000000006
:101AE000000000000000000000000077000000007F
:101AF00003B800000000000000000000000000002B
:101B000000000000000000000000000000000000D5
:101B100000000000000000000000000000000000C5
:101B2000000000000000000078000000000000003D
:101B300000000000000000000000000000000000A5
:101B40000000000000000000200000000000000075
:101B500000000000003801C03E07F00003C0000094
:101B600000007003807C00070FF000001FC03800E9
:101B7000E01F01FC00000000001C003807C000004E
:101B8000E000000000E39C18C7F078700FC0E1CEC1
:101B900006000000000E3F00703F07F00707F83F07
:101BA0008FFC7F83F00000000000000FE00FF801C1
:101BB000F01FF80FE07FC0FFE3FF03F8381CE01CC4
:101BC000383E7007E3F3C1C1FE07FE07F81FF80FA8
:101BD000E1FFCE07783FC3E1FE07F01EFFE7F8F80C
:101BE0001E0001C0001C0000000E0001F0003801C2
:101BF000CE700700000000000000000000000000A0
:101C00000000000000000000001E6780000000FED1
:101C1000FC001F800000000380383E78E0007F0059
:101C20000FDFFDF9FFFF7E19C318E7000000000079
:101C30003F9FBCF03E00000007E1F1C0780000309B
:101C40007E0003C78C1F8C61FC3F8000000007F002
:101C50000003E0707C7C70003FF000061F0000C0B5
:101C60007030383E07000007C00F801F003E007C28
:101C700000F801FFFC1FC0FFE3FF8FFE3FF9CE71AC
:101C8000C3FE0F0707F807F807F807F807F8000082
:101C90007FFB81CE07381CE07701E7001FC01C03E3
:101CA000803E07F06303C0000000003807007C0C92
:101CB000639DF461F81FC01C01C01F01FC0C600093
:101CC00000000E007007C06301C0E0031800E39C31
:101CD00039CFF8FC701FE0E1CE06000000000E7F57
:101CE00080F0FF8FF80F07F87FCFFCFFC7F80000E8
:101CF000000000001FF01FFE01F01FFC1FF87FF026
:101D0000FFE3FF0FFE381CE01C387C7007E3F3C1D3
:101D1000C3FF07FF0FFC1FFC1FF1FFCE07783FC377
:101D2000E1EF0F783CFFE7F8F81E0000E0001C0030
:101D300000000E0003F0003801CE70070000000024
:101D40000000000000000001000000000000000092
:101D500000003E67C0000001FEFC001F8000000084
:101D60000380383EFCE000FF801FFFFDF9FFFF7E8F
:101D700039C738E700000000003F9FBCF03E00007C
:101D80000007E1F1E0F0000030FF8003C78C3FCC9A
:101D900067FF3F800000001FFC0007F070FCFCE0C4
:101DA000007FF0001E3F8003C0E0F0387E0E000090
:101DB00007C00F801F003E007C00F801FFFC3FF0D1
:101DC000FFE3FF8FFE3FF9CE71C3FF0F070FFC0F3C
:101DD000FC0FFC0FFC0FFC0000FFF381CE07381C4A
:101DE000E07783C7003FE01C03807705F06303C002
:101DF00000000000380700EE0C639DBC60F017C0C7
:101E00001C01C03B817C0C600000000E00700EE0E5
:101E10006301C0E0031800E39C39CFFCFC701FE0B5
:101E2000E3CF3FC1C000000EF3C1F0F3CF781F072E
:101E300080FBC03CF3CF7C0000030003003EF83E73
:101E40003F03F81FFC3FFC7FF0FFE3FF1FFF381C40
:101E5000E01C38F87007E3F3E1C7FF87FF1FFE1FA0
:101E6000FC3FF9FFCE07783FC3E1E79E3C78FFE7F0
:101E7000F8F83F0000E0001C0000000E0003C00066
:101E800038000070070000000000000000000000A3
:101E900007000000000000000000003E67C0003F97
:101EA000E3FEEC003C0000000003803877FCE0011A
:101EB000FFC01FFFFDD9FFFB7621C420E700000013
:101EC00000002F863CF000000000076000F1E000F9
:101ED0000031E78001EF0C3FC00F8F8380000000CE
:101EE0003E3E00077070ECFCE0007E60001E3B8010
:101EF00003C1C0F0707E0E00000FE01FC03F807F66
:101F000000FE01FC03DFFC7FF8FFE3FF8FFE3FF9DB
:101F1000CE71C3FF8F871FFE1FFE1FFE1FFE1FFE19
:101F20000001FFE381CE07381CE073C787003DE066
:101F300000000000000000000000000000000000A1
:101F4000000000000003F800000000000000000096
:101F5000003800000000000000000000E000000069
:101F6000E39C39CEDCCCE01CE0E3873FC1C000003D
:101F70000CF3C7F0E1CE381F0780F18038E1CF3C89
:101F800000000F0003C03C78780703F81C3C7E7CFF
:101F900071F8E003801F1F381CE01C39F07007E364
:101FA000F3E1CFCFC70F3F3F1C3C3CF81C0E073C72
:101FB0007BC7F1E79E3C7801E738383F000000001E
:101FC0001C0000000E0003800038000070070000B5
:101FD00000000000000000000007000000000000FA
:101FE000000000003C63C0003067E6EC003C0000ED
:101FF00000000383FF80CDC001E7C03E7C01D80311
:10200000FB7638473821000000000000063FF00052
:10201000000000076000F1E0000021E78C61EF0C98
:102020003DC00E039F80000000380E000630701C7B
:102030003C00007E60001E318003C1C0F0E01E1C29
:1020400000000FE01FC03F807F00FE01FC03DC00AA
:10205000FCF8E003800E003801CE71C387CF873FC4
:102060003F3F3F3F3F3F3F3F3F1873F3F381CE0772
:10207000381CE073C787FE38E00000000000000055
:102080000000000000000000000000000000033815
:102090000000000000000000000038000800000000
:1020A0000000000000E0000000E39DFFEEC0CCE077
:1020B0001FE0E787BFC1C000001CF3C7F001C038B4
:1020C0003F0F00E00078E1CE1C70E07F3FF3F800A6
:1020D00038E7FB83B81C1C783C7078E003803C0F29
:1020E000381CE01C3BE07007F7F3F1CF03C7073C57
:1020F0000F1C1C38781C0E073C79E7F1C3FC1EF05E
:1021000003C71C387F800000FF1DF03F03EE1F8FC8
:10211000E1F73BF1CE71E73BEFC77E0FE1DF03FE56
:102120007F3FCFCE0EF07F1C7F0FE0E7FC3861C011
:1021300000306780EC00FF000000003FFBFF80CD17
:10214000C001C3C3BC3C01D807BB7639C738E70020
:1021500000000000000637B0FF1C0FEFC767FC7BD4
:10216000C00707F1C01FF0EE0C3E001CF1FF8739DD
:10217000FF8073E7000777FF381C03877E60000647
:1021800031B9C0C38030E00E3800E00EE01DC03B26
:10219000807700EE01DC079C00F078E003800E0001
:1021A0003801CE71C383CFC73C0F3C0F3C0F3C0FAF
:1021B0003C0F3CF3C3F381CE07381CE071EF07FFFF
:1021C00039E0FF0FF0FF0FF0FF0FF0FFFC0FC0FC36
:1021D0000FC0FC0FC39CE383FC77E0FE07F03F8158
:1021E000FC0FE03807FCE0E7073839C1DC1CEF8E54
:1021F0000E00E001FFEFC0FDC01FC007879F81C038
:1022000000001CE1C77003C0F87F0FF0FF00F0F37F
:10221000CE1C70E1FF3FF3FE0078EFFB87BC1C3C57
:1022200078007078E003803C00381CE01C3BC070F4
:1022300007F7F3F9CF03C70F3C0F1C3C3E001C0E01
:10224000073C79E773C1F80FE007871C38738000FB
:1022500001FF9FF87F87FE3FCFE3FF3FF9CE73C7B3
:102260003FFFE7FF1FF1FF87FE7F7FEFCE0E78F77E
:102270003E779EF1E7FC3861C000306FFCEC00FF58
:10228000000000003FFBFF80FF8001F003BC3FF92E
:10229000D80F3B76398738C61E000000000006378D
:1022A000B1FF9C1FFFE767FC3F80070FF9E03FF895
:1022B000FE0C3F001DF9FB8739FF8073670007F7AD
:1022C000FF70FC03877E6000063BB9C0C78031C049
:1022D0007E3800E01EF03DE07BC0F781EF03DE07B3
:1022E0009FF8F000E003800E003801CE71C383CF69
:1022F000E73C0F3C0F3C0F3C0F3C0F3FF3C7F38113
:10230000CE07381CE070FE07FF39E1FF9FF9FF9F01
:10231000F9FF9FF9FFFE1FE1FE1FE1FE1FE39CE3B3
:1023200087FE7FF1FF0FF87FC3FE1FF0000FF8E07C
:10233000E7073839C1DE3CFFCF1E00E000738FF0A5
:10234000FDC00F8007879F9FFC00001CE1C670073F
:10235000C1F0770FF8FF80E07F8F3C70E3F83FF02B
:102360007F00F9DFFB87BC1FFC70007038FFC3FEE5
:1023700038003FFCE01C3FC07007F7F3B9CE01C73F
:10238000FF38071FFC3FE01C0E071C71EF7BC1F8F4
:102390000FE00F071C38F3C00001C79F7CFBCFBEC6
:1023A00079E387DF3E79CE77873EFDE7CF3EF9F7C9
:1023B000CFBE7979E70E0E78F7BEF3FCF1E03C383A
:1023C00061C7F3306FFCEC003C000000003FF838C0
:1023D00000FF8001FF07381FF9D81E3B7600000080
:1023E000003F00000000000637B1E78E3EFCF760BA
:1023F0003C3F80071FFDE03EF8FE0C7FC01980FFC8
:102400008E71FF8063630003E7FFFCFC03877E633C
:1024100080063F9CE0C70031C07E7000E01EF03DAA
:10242000E07BC0F781EF03DE071FF8E000FFC3FF8A
:102430000FFC3FF1CE71CFF1CEE7380738073807F0
:10244000380738071FE38F7381CE07381CE070FE12
:10245000070F39C1C79C79C79C79C79C79C7CF3E04
:10246000F3CF3CF3CF3CF39CE38FBE7CF3EF9F7C38
:10247000FBE7DF3EFBFF9F7CE0E7073839C1DE3C2E
:10248000FBEF1E00E0007387FC7B803F8007039911
:102490009FFC000018E1C0700F81F8E70F7CF3C1CA
:1024A000E07F8F3C0003C000000F01F1DFF18F1EC1
:1024B0001FFC70007038FFC3FE387F3FFCE01C3FFC
:1024C000E07007F7F3BDCE01C7FE38071FF81FF015
:1024D0001C0E071EF1EF7BC0F007C01E070C38F37F
:1024E000C000003F9E3CF3CF1E70E3878F3C39CE87
:1024F0007F073C78E78F3C79E3CF1E7878070E0E94
:1025000038E3BEE1F871C0787861E7FF306700EC2E
:10251000003800000000038038007B8000FF8F3807
:102520001FF9D83C3B76000000003F00000000008F
:10253000063331E00F3C7C7760781F00001EFFFC03
:102540001C71FF0C7FE01980FF9EF0038063E300A5
:10255000000070FC7803873E6380061F1EF0CE1CCF
:10256000339F3CE1C0003C7878F0F1E1E3C3C787DA
:102570008F0F1FF8E000FFC3FF0FFC3FF1CE71CFBC
:10258000F1CEF7380738073807380738070FC39EEA
:102590007381CE07381CE0707C070739E03F83F871
:1025A0003F83F83F83F803C73CF38738738738735A
:1025B0009CE38F1E78F3C79E3CF1E78F3C7BFF9E28
:1025C0007CE0E7073839C1CE38F1E71C00E0007342
:1025D00081FC03BC7FFC0703801FFC07E038E1C0DF
:1025E000700F817CC7003CF3C1E0F3C7FC0003F827
:1025F00000007F03C1DEF18F1E1FFE70007038FFE8
:10260000C3FE387F3FFCE01C3FE07007FFF39DCE28
:1026100001C7FC38071FF007F81C0E071EF0EE3B41
:1026200081F807C03C070E3800000000FF9C1CE04A
:102630000E0E7FE387073839CE7F073870E70738FB
:1026400039C1CE0E707F070E0E3DE3BEE1F87BC0B0
:10265000F07861E7FF306FF8EC00780000000003CD
:102660008038000778F03FCE381C01D8783B7600E0
:102670000000003F0000000000000001FC07383FA0
:10268000F760F01F00071CC3FC1831FF0C73E01942
:1026900080C01CE0039FE3E300000070000003879C
:1026A00006638000000E700E3C073F00E3C0E03C74
:1026B0007878F0F1E1E3C3C7878F0FFC00E000FFFB
:1026C000C3FF0FFC3FF1CE71C381CE7738073807C7
:1026D0003807380738070FC3BC7381CE07381CE0B2
:1026E000707C070F39F0FF8FF8FF8FF8FF8FF83FEE
:1026F000FF3803FF3FF3FF3FF39CE38E0E707383BD
:102700009C1CE0E707383BFF9CFCE0E7073839C139
:10271000CF78E0E7BC00E001FFE0FC077E7BFC0730
:10272000038001C007E038E1C0701F003DC7001CF6
:10273000E1C3C0F3C3FC0001FF3FF3FE03C19CF300
:102740008FFE1C1E78007078E003803C7F381CEE02
:102750001C3CF07007FFF39FCF03C7003CEF1CF059
:1027600000F81C0E070FE0FE3F81F8038078070E8B
:102770003800000001FF9C1CE00E0E7FE387073845
:1027800039CE7F873870E7073839C1CE0E703FC722
:102790000E0E3DE3FFE0F07BC1F0F060F67F306F9E
:1027A000F8EC0078000000000380380007FDF8070F
:1027B000CE3C3C01D8F03B76000000003F7FFFFF9D
:1027C000FFC0000000FF07383FF761F00E00071C54
:1027D00080E01C70380079E01DF9C01CE0039FF315
:1027E00077000000700000038706600000000E7094
:1027F0001C6C073B01C6C1E03FF87FF0FFE1FFC35F
:10280000FF87FF1FFC00F000E003800E003801CEC0
:1028100071C383CE7F3C0F3C0F3C0F3C0F3C0F1F1E
:10282000E3F8F381CE07381CE0703807FF38F9FF72
:102830009FF9FF9FF9FF9FF8FFFF3803FF3FF3FF6A
:102840003FF39CE38E0E7073839C1CE0E7073838DF
:10285000001DDCE0E7073839C1CF78E0E7BC00E0D5
:1028600001FFE0DC077E71FC07038001C007E03850
:10287000F3C0703E001DFFC01CE1C3C0E1C01C00DE
:10288000007F3FF3F803819DF39FFF1C0E783C709F
:1028900078E003803C07381CEF1C38F07007BEF36B
:1028A0008FCF03C7003CFF1C7878381C0F0F0FE058
:1028B000FE3F83FC0380F0070E3800000001E39C1C
:1028C0001CE00E0E700387073839CE7F873870E71B
:1028D000073839C1CE0E701FE70E0E1FC3F7E1F89F
:1028E0003F81E0F060F000306780EC00780000008D
:1028F000000380380006FDFBC1CF3C3C01D9E03B22
:1029000076000000001E7FFFFFFFC00000007F8FE9
:1029100038380761E00E00071F81E03EF9FF007CB8
:10292000E01CF1C01EF0039FF37700000070000070
:10293000038706600000001EF038CC0E07038CC32E
:10294000E07FFCFFF9FFF3FFE7FFCFFF9FFC00F004
:1029500078E003800E003801CE71C383CE3F3C0F78
:102960003C0F3C0F3C0F3C0F3FF3F0F3C3CF0F3C49
:102970003CF0F03807FE3879E39E39E39E39E39E58
:1029800039FF8038038038038038039CE38E0E7053
:1029900073839C1CE0E7073838381F9CE0E7073852
:1029A00039C1C7F0E0E3F8000000E70EDC0766710C
:1029B000F807038001C0000070F3C070780F3DFF7E
:1029C000CF3CF3C3C0F3CE3C00000F3FF3C0000187
:1029D0009FF71FFF1C1E7E7C70F8E003801F1F38CE
:1029E0001CEF3C38787007BEF387CFCFC7003FFF9E
:1029F0001C3C7CF81C0F9F0FE0FE1F879E0381E0AC
:102A000007063800000001C79E3CF3CF1E79E3871C
:102A10008F3839CE73C73870E7073C79E3CF1E7023
:102A200001E70F1E1FC1F7C3F83F83C07861E000C4
:102A30003067E6EC007800000000038038000ECD1F
:102A40009BE7C73E7C01DBC03B7600000000000036
:102A500000000000000000078E3C7CF763C00E0001
:102A6000071FBDE03FF9FF007FE00E03800E7003FB
:102A700080380E00000000000003CF066000000058
:102A80001CE038FE0E0E038FE7C07FFCFFF9FFF35A
:102A9000FFE7FFCFFFBC1C00FCF8E003800E00380E
:102AA00001CE71C387CE1F3F3F3F3F3F3F3F3F3F78
:102AB0003F3CF3F3F3E7CF9F3E7CF9F03807FC3857
:102AC00039C79C79C79C79C79C79C3CF3CF3CF3C6D
:102AD000F3CF3CF39CE38F1E7073C79E3CF1E78FEE
:102AE0003C78381F3CF1E78F3C79E3C7F0F1E3F81D
:102AF00000E000E70FFC0E6679FC07878001C1C08B
:102B00000E70F3C070F00F3C070F7CFBC3C0F3CF17
:102B10007C70E0030003000381DFEF1C071FFE3F12
:102B2000FC7FF0FFE3801FFF381CEFFC383C7FE7A1
:102B30003E7387C7FF87001FFE1C3C7FF81C0FFFFA
:102B400007C07C1F079E0381FFE7073800000001D4
:102B5000EF9F7CFBCFBE7DE387DF3839CE71E7384E
:102B600070E7073EF9F7CFBE7079E70F3E0F81F7A8
:102B7000C3FC1F07807861E0003063FEECE0783929
:102B8000C3870E038038000ECD9BFFC39FFFFDDB84
:102B9000FFFB7600000000000000000000000001C4
:102BA000E79C3EFEF767800E00071FFFFF9FF0388F
:102BB0000C3FC00F8F80073800003E3E000007FF2B
:102BC000000003DF066000000039C070FE1C1C0717
:102BD0000FEF80701CE039C07380E701CE03BC1F8B
:102BE000FC7FF8FFE3FF8FFE3FF9CE71C3FF8E1F1E
:102BF0001FFE1FFE1FFE1FFE1FFE3871FFE3FFCFEB
:102C0000FF3FFCFFF03807003BF9EF9EF9EF9EF91C
:102C1000EF9EF9EFEF3EF3EF3EF3EF3EF39CE38FD1
:102C2000BE7073EF9F7CFBE7DF3EF8381F7CF3E755
:102C30009F3CF9E7C3E0FBE1F000E000E70FF80E8E
:102C40007E3FFE0787800001C00E707F8070FFC747
:102C5000F80707F87F83807F8FF870E0000000009E
:102C60000381DFFE3C079FFE1FF87FF0FFE3800F2C
:102C7000FE381CE7F8383C7FE73E7383C3FF07004C
:102C80000FFF9C1E3FF01C07FE07C07C1F0F0F03A9
:102C900081FFE7073800000001FFDFF87F87FE3F74
:102CA000C383FF3839CE71E73870E7071FF1FF871C
:102CB000FE707FE7CFFE0F81F7C79E1F07FC3861CC
:102CC000C0003061FEECE07039C3870E0383FF80E3
:102CD0001CFDF9FF839FFFFDDBFFFB76000000007A
:102CE000000000000000000001FF9C1FFFE767FCE0
:102CF0000E00070FFBFF8C60380C0FC007FF0007AA
:102D00003800001FFC000007FF000003FF06600002
:102D1000000039C0E00C383F0F00CF00F01FE03F4B
:102D2000C07F80FF01FE03F81FFC3FF0FFE3FF8F31
:102D3000FE3FF9CE71C3FF8E0F0FFC0FFC0FFC0F8F
:102D4000FC0FFC0003FFC1FF87FE1FF87FE0380780
:102D5000003BF9FFDFFDFFDFFDFFDFFDFFFE1FE1B1
:102D6000FE1FE1FE1FE39CE387FC7071FF0FF87FFD
:102D7000C3FE1FF0000FF8FFE7FF3FF9FFC3E0FFBE
:102D8000C1F000E000E707F81C7E1FDC0787800029
:102D900001C00E703F0070FFC3F00703F03F0380D7
:102DA0003F07F070E0000000000381CEF83C079F71
:102DB000FC0FE07FC0FFE38003FC381CE3F0381E0B
:102DC0007FE73E7383C1FE070007FF9C1E1FE01CC8
:102DD00003FC07C07C1F1E078381FFE70738000044
:102DE0000000FFDDF03F03EE1F8381F73839CE701E
:102DF000F73870E7070FE1DF03EE703FC7C7EE0754
:102E000000E38F0F1F07FC3861C0003FE0FEFCE0CD
:102E1000F039C3870E0383FF801CFDF8FF000FFF0E
:102E2000FDFBFFFF7E00000000000000000000002E
:102E30000000FF000FEFC7E7FC0E000707F3BF809D
:102E400000380C07C001FC000000000007F0000083
:102E500007FF000003FF06600000000000E00C38E0
:102E60003F0E00CE00F01FE03FC07F80FF01FE0359
:102E7000F81FFC1FC0FFE3FF8FFE3FF9CE71C3FEBA
:102E80000E0F07F807F807F807F807F80007FF80A4
:102E9000FF03FC0FF03FC038070039F0FFCFFCFF05
:102EA000CFFCFFCFFCFEFC0FC0FC0FC0FC0FC39C8F
:102EB000E383F87070FE07F03F81FC0FE0001FF025
:102EC0007EE3F71FB8FDC3E0EF81F00000000000D3
:102ED000C01C3C0000038700000040000000000010
:102EE00000000000000000000000000000200000C2
:102EF00000000000E003C00000000000000000002F
:102F000000000000000000000000000000000000C1
:102F1000000000038000000000000000000000002E
:102F20000000000007003800000000000000000062
:102F3000000000000700000E00000000000000017B
:102F4000C0000E000000000000000000001E000095
:102F50003C63C0000000000020F008400000038334
:102F6000FF801C78F000000000000000000000005E
:102F70000000000000000000000000000000000051
:102F800000000000070200000000000C39C0000033
:102F900000000000000000000000000000038006A8
:102FA000600F800000000000000000000F1E000005
:102FB0000000000000000000000000000F80000082
:102FC0000000000000000000000000000000000001
:102FD00000000000000001000000000000000000F0
:102FE00000000000000000000000000000000000E1
:102FF00007C000000000000000000000000000000A
:1030000000000000000000080000000000000003B5
:10301000C0E001E00000000000C00000000003C7A5
:10302000000001C0000000000000000000000000DF
:10303000000000000000E0000000000000F007C0F9
:103040000000000000000000000000000000000080
:103050000000000000000000000000000000000070
:103060000000000000000000000000000007C0F8A1
:10307000000000000000000000000000079F0000AA
:103080001E0000000000000001C0000E0000000053
:103090000000000000001E00003E67C000000000AD
:1030A00000E0F039C000000380380000000000009C
:1030B0000000000000000000000000000000000010
:1030C00000000000000000000000000000070600F3
:1030D000000000000C3FC0000000000000000000E5
:1030E000000000000000038006600B80000000006C
:1030F00000000000000FBE00000000000000000003
:1031000000000000000B8000000000000000000034
:1031100000000000000000000000000000000000AF
:10312000000000000000000000000000000000009F
:1031300000000000000000000005C00000000000CA
:10314000000000000000000000000000000000007F
:10315000000000000000000003C0E001E0000000EB
:103160000000000000000001CE000001800000000F
:10317000000000000000000000000000000000C08F
:103180000000000000007E3F800000000000000002
:10319000000000000000000000000000000000002F
:1031A000000000000000000000000000000000001F
:1031B00000000000000007C0F8001FFE0000000033
:1031C000000000000007FF00001E000000000000DB
:1031D0000001C0000E000000000000000000007CA4
:1031E00000003E67C00000000000C7F03180000012
:1031F0000380380000000000000000000000000014
:1032000000000000000000000000000000000000BE
:10321000000000000000070600000000000C3FC096
:10322000000000000000000000000000000000039B
:10323000800660038000000000000000000007FC22
:1032400000000000000000000000000000000380FB
:10325000000000000000000000000000000000006E
:10326000000000000000000000000000000000005E
:10327000000000000000000000000000000000004E
:10328000000001C00000000000000000000000007D
:10329000000000000000000000000000000000002E
:1032A000000F80E007C000000000000000000000E8
:1032B00001CE00000000000000000000000000003F
:1032C0000000000000000000000000000000003FBF
:1032D000FF000000000000000000000000000000EF
:1032E00000000000000000000000000000000000DE
:1032F00000000000000000000000000000000007C7
:10330000C0F8001FFE00000000000000000003FCE9
:1033100000001C0000000000000001C0000E0000C2
:1033200000000000000000007C00001E678000001C
:1033300000000007E00000000003803800000000EB
:10334000000000000000000000000000000000007D
:103350000000000000000000000000000000000766
:103360000600000000000C1F8000000000000000AC
:103370000000000000000000038006601F800000C5
:103380000000000000000003F80000000000000042
:10339000000000000000001F80000000000000008E
:1033A000000000000000000000000000000000001D
:1033B000000000000000000000000000000000000D
:1033C00000000000000000000000000FC00000002E
:1033D00000000000000000000000000000000000ED
:1033E000000000000000000000000F80E007C000A7
:1033F00000000000000000000000000000000000CD
:1034000000000000000000000000000000000000BC
:1034100000000000000000000FFC000000000000A1
:10342000000000000000000000000000000000009C
:10343000000000000000000000000000000000008C
:10344000000000000000000000000000000000007C
:10345000000000000000000000000000000000006C
:10346000000000000000000000000000000000005C
:1034700000000000006000000000000000000000EC
:10348000000000000000000000000000000000003C
:10349000000000000000000000000000000000002C
:1034A0000000000000000000000000000000000C10
:1034B000000000000000000000000000000000000C
:1034C00000000000000000000000000000000000FC
:1034D00000000000000000000000000000000000EC
:1034E00000000000000000000000000000000000DC
:1034F00000000000000000000000000000000000CC
:1035000000000000000000000000000000000000BB
:1035100000000000000000000000000000000000AB
:10352000000000000000000000000000000000009B
:10353000000000000000000031C397206D69747422
:10354000696720616E74697070656E2100426974EC
:10355000746520616C6C652076696572204B7265BC
:10356000697365006B616C696272696572656E0092
:10357000546F75636873637265656E0053656B2E77
:10358000004D696E2E005374642E00546167004D27
:103590006F6E2E004A61687200446174756D2F551C
:1035A00068727A656974207374656C6C656E002549
:1035B0006400536F004D6F004469004D6900446F13
:1035C00000467200536100002564002553006272BA
:1035D00061756E00626C6175006772617500676588
:1035E0006C6200255320323025303264004D6F6EFE
:1035F0006174736B616C656E64657200005550AAEE
:10360000A0A590FFF0F5D0FAE0E5E4000130112428
:103610001FBECFEFD8E0DEBFCDBF13E0A0E0B1E02A
:10362000ECE0FAE702C005900D92A034B107D9F79B
:1036300014E0A0E4B3E001C01D92A53EB107E1F79C
:1036400016E3CEE0D6E304C02297FE010E94003DBF
:10365000CC30D107C9F7F4D40C9458390C9400003D
:10366000FC018F3F910509F048F48031910518F075
:1036700084E090E00CC080E090E009C080E1E030A0
:10368000F80718F08CE090E002C088E090E020E1BC
:1036900030E0281B390B02C0F695E7958A95E2F7D2
:1036A000E05CFE4F8081281B3109C9010895EE2797
:1036B000FF27E81BF90BE823F923EF3FF10509F099
:1036C00048F4E031F10518F024E030E00CC020E0CF
:1036D00030E009C080E1E030F80718F02CE030E07D
:1036E00002C028E030E0022E02C0F695E7950A9469
:1036F000E2F7E05CFE4F808121503040280F311D01
:10370000C9010895292FA0E4B2E0FD01E80FF11DE1
:10371000808130E0A20FB31F2C9130E0280F311DC3
:10372000C90108959C014091420350914303809147
:103730004A0390914B03481B590B460F571F80E4D7
:1037400093E0B9010C94C4230F931F93CF93DF939D
:10375000EC01109249031092480310924B0310920F
:103760004A038091640380FD28C000E411E020EF4B
:1037700030E0235030400350104080E493E062E09A
:1037800070E043E150E065D7D0936A03C0936903CA
:10379000809165038D7F8093650380E493E0BE0193
:1037A0000E94CD29C095D095D0936803C09367033C
:1037B000DF91CF911F910F91089500EF10E020E469
:1037C00031E0D7CFCF92DF92EF92FF920F931F930A
:1037D0007C016901D9D7C701B601A8010E94FB2766
:1037E0001F910F91FF90EF90DF90CF900895CF92AF
:1037F000DF92EF92FF920F931F937C016901C4D770
:10380000F70185A1806185A3C701B601A801E5D7AD
:10381000C7010E940D24C7010296FFD7C7010E946D
:1038200088261F910F91FF90EF90DF90CF90089521
:103830008F929F92AF92BF92CF92DF92EF92FF92C0
:103840000F931F934C015B0197E6C92E93E0D92E8D
:1038500084E195EA909368038093670390936A03E9
:1038600080936903F601329780818D7F808389ED93
:103870009FEFC80ED91EC60160E070E040E050E046
:1038800020EF30E08401B3DF80E4E82E81E0F82E01
:10389000A7014A195B09C60160E070E020EF30E043
:1038A0008501A5DFE818F908EA18FB08C60160E001
:1038B00070E0A40122E030E0870199DFC6016EEEDE
:1038C00070E0A40122E030E092DF109268031092D1
:1038D0006703C6016FE572E00E94272C82E08093A7
:1038E00066031F910F91FF90EF90DF90CF90BF90F4
:1038F000AF909F908F900895AF92BF92CF92DF923A
:10390000EF92FF920F931F93CF93DF9383E190E0A9
:1039100062E070E08DDF80E493E068E770E040E013
:1039200050E032D780E493E06EEC70E00E94FB2B15
:103930008FEF9FEF09DF1092490310924803109216
:103940004B0310924A0380E090E0FEDEFEEDAF2EC6
:10395000F0E0BF2E6501CAEAD0E0F60185919491AE
:10396000909368038093670340E451E04C1B5D0B28
:103970000CE711E00C1B1D0B80E493E0BE01EC96FC
:103980009E01E6E0EE2EF12C0E94992882E090E064
:10399000C80ED91EC055D04098EEC91690E0D90681
:1039A000E1F6C8E2D0E0F501859194919093680327
:1039B0008093670380E493E0BE01EC96AE012EE1B4
:1039C00030E00E94432982E090E0A80EB91EA8973B
:1039D00098EEA91690E0B90631F780E098EF909341
:1039E000680380936703E0905E03F0905F0380912B
:1039F0005A0390915B03E81AF90AC0E0D0E015C0C1
:103A0000609158037091590340915A0350915B03A0
:103A10004C0F5D1F9E01260F371F00915E03109112
:103A20005F0380E493E0CEDE2A96CE15DF0544F3F3
:103A3000E70115C000915A0310915B0360915C038C
:103A400070915D03AE01400F511F209158033091DA
:103A500059032C0F3D1F80E493E0B4DE2A971C1617
:103A60001D0644F38FEF97E09093680380936703FC
:103A7000E70115C000915A0310915B036091580350
:103A800070915903AE01400F511F20915C0330919A
:103A90005D032C1B3D0B80E493E094DE2A971C16FB
:103AA0001D0644F3C0E0D0E015C060915C03709146
:103AB0005D0340915A0350915B034C0F5D1F9B01C6
:103AC0002C1B3D0B00915E0310915F0380E493E09B
:103AD00079DE2A96CE15DF0544F3DF91CF911F9151
:103AE0000F91FF90EF90DF90CF90BF90AF9008952F
:103AF000809113018F5F809313018C33C1F4109276
:103B00001301809114018F5F809314018C3379F439
:103B100010921401809115018F5F809315018831F7
:103B200031F41092150186E191E00C94892F0895EB
:103B30001F920F920FB60F9211242F933F934F9322
:103B40005F936F937F938F939F93AF93BF93EF9305
:103B5000FF93CEDFFF91EF91BF91AF919F918F9136
:103B60007F916F915F914F913F912F910F900FBE79
:103B70000F901F901895EF92FF920F931F93DF9372
:103B8000CF93CDB7DEB76497DEBFCDBF8DB79EB7FD
:103B90000A979EBF8DBFEDB7FEB731967E010894A0
:103BA000E11CF11CADB7BEB71296FC92EE921197D4
:103BB00088EE90E09383828380911501992787FD99
:103BC00090959583848380911401992787FD909522
:103BD0009783868380911301992787FD909591871C
:103BE00080870E9463398DB79EB70A969EBF8DBFAE
:103BF00000E413E0C80168E770E042E251E0C4D598
:103C0000C801B7010E94AB2B6496DEBFCDBFCF9138
:103C1000DF911F910F91FF90EF900895EF92FF9227
:103C20000F931F93CF93DF93EC0148815981411586
:103C30005105E9F08C819D8190936803809367031F
:103C40004B5050400A811B81055F1F4F80E493E079
:103C500065E070E02BEE30E0AAE0EA2EF12C0E9445
:103C600072278C819D81809590959D838C83DF91B7
:103C7000CF911F910F91FF90EF9008950F931F9395
:103C8000CF93DF938C01EB01209741F0C8010E9494
:103C90005A390196080F191F2197F6CFC801DF91F5
:103CA000CF911F910F910895EF92FF920F931F9361
:103CB000DF93CF93CDB7DEB76497DEBFCDBF09E604
:103CC00013E010926A0310926903F801349780811F
:103CD0008D7F80838FEF9FEF9093680380936703BE
:103CE00086E191E00E94202F682F772767FD70956D
:103CF00089EF90E0C3DF00D000D000D0EDB7FEB771
:103D000031967E010894E11CF11CADB7BEB7129646
:103D1000FC92EE92119727E431E03383228395835E
:103D200084830E9463392DB73EB72A5F3F4F3EBF61
:103D30002DBF09521040C80168E770E040EF50E025
:103D400023D5C801B7010E94AB2B609117017727DB
:103D500067FD7095615070408AE790E08FDFADB7E6
:103D6000BEB71C97BEBFADBFEDB7FEB7319612967A
:103D7000FC92EE92119727E331E033832283209166
:103D80001601332727FD3095358324839783868357
:103D900080911901992787FD90959187808780915F
:103DA0001801992787FD9095938782870E94633930
:103DB0002DB73EB7245F3F4F3EBF2DBFC80168E718
:103DC00070E049E051E0E0D4C801B7010E94AB2B9C
:103DD0006496DEBFCDBFCF91DF911F910F91FF9011
:103DE000EF9008952F923F924F925F926F927F9241
:103DF0008F929F92AF92BF92CF92DF92EF92FF92FB
:103E00000F931F93DF93CF9300D000D0CDB7DEB7D1
:103E1000882E8091160190911701A0911801B09100
:103E2000190189839A83AB83BC8310E005C0CE015E
:103E300001960E94892F1F5F1815CCF310E099247A
:103E400001E0CE010196612F0E944E348111902A2B
:103E50001F5F143011F0000FF4CF992011F410E01F
:103E600005C0892D90E023DC182F1F5F292C3324F7
:103E7000C10148DC082F882309F401E0812F99272C
:103E800087FD9095880F991FFC01E859FF4F4590D9
:103E90005490FC01E45BFE4F65907490509268036F
:103EA00040926703C0904203D090430380914A033D
:103EB00090914B03C81AD90A82E290E0C80ED91E2D
:103EC00084E1080250011124AC0CBD1C8EED9FEF63
:103ED000C80ED91E91E0891699F4992069F0D09204
:103EE0007503C0927403B0927703A0927603709228
:103EF00079036092780304C01092750310927403E2
:103F000080E493E060E170E0A60120EE30E08501FE
:103F1000E6E0EE2EF12C0E949928709268036092E0
:103F2000670380E493E060E170E0A60120EE30E0FA
:103F3000B3E0EB2EF12C08D750926A03409269034C
:103F4000809165038D7F8093650384E090E0C80EC7
:103F5000D91E80E493E06EE170E0A60115D4682DCF
:103F6000772767FD70958BE991E088DEBC0180E4DE
:103F700093E00E94FB2B8EE190E068E170E0D2DBE1
:103F80009920C1F110E8EE24FF24812F90E08221D6
:103F90009321892B31F1123079F0133018F411305C
:103FA000D9F405C0143069F01830B1F40FC080E4C2
:103FB00093E06FE871E00EC080E493E063E871E0A5
:103FC00009C080E493E067E771E004C080E493E017
:103FD0006AE671E00E94FB2B8EE190E064E170E004
:103FE000A1DB16950894E11CF11C98E0E916F10498
:103FF00061F60BC080E493E06EE571E00E94FB2B5C
:104000008EE190E064E170E08DDB80E190E063E1BF
:1040100070E088DB2496DEBFCDBFCF91DF911F918A
:104020000F91FF90EF90DF90CF90BF90AF909F9057
:104030008F907F906F905F904F903F902F9008955A
:10404000EF92FF920F931F93DF93CF9300D000D096
:10405000CDB7DEB78AE793E060E070E040EC50E077
:104060000E94523B80E493E060E00ED583E793E04A
:104070000E946A2C109280008DE08093810088E07D
:104080009DE3909389008093880082E080936F0085
:1040900081E083BF86EF809364007894CE0101961F
:1040A00060EC70E044E050E00E94523B8AE394E010
:1040B0006CEC70E048E050E00E94523B898188310E
:1040C000C0F58A8181508F31A0F58B8181508C3071
:1040D00080F58C81843668F589819A81AB81BC81B9
:1040E0008093150190931601A0931701B0931801C6
:1040F000109214010BEC10E0B8E0FB2E13C0C801C5
:104100000E94623B809501501040882359F090E056
:10411000A7DA90E1981BFF0CFF0CFF0C9F0D90930A
:10412000140104C0FA942FEFF21649F787E3809345
:104130001301E0901401FF240E2D10E08091140172
:10414000992787FD90950817190709F43EC085E166
:1041500091E060EC70E044E050E00E946A3B4091E6
:104160001401442399F424EC30E0F999FECF32BDD8
:1041700021BDF89484E18FBB86E18FBB78942F5FDB
:104180003F4F80E02C3C380781F71DC0F999FECFE6
:10419000C801A3E095958795AA95E1F78C539F4FA9
:1041A00092BD81BD0770107081E090E002C0880F61
:1041B000991F0A95E2F7809580BDF89484E28FBB41
:1041C00086E28FBB78941FBAE42E409116012F2D02
:1041D00030E0842F992787FD909528173907D9F06B
:1041E000F42E8ADB80E493E06CE775E10E94272CD3
:1041F0001092660380E493E060E170E049E150E0F2
:10420000C3D280E0EFDD81E0EDDD82E0EBDD82E036
:104210008093660349DD83E793E00E947E2C882328
:10422000A9F183E793E060E90E94832C80509240DB
:104230005CF40E946F2D882321F18AE394E06CECFA
:1042400070E048E050E012C083E793E060ED0E9428
:10425000832C80509240B8F40E942436882349F081
:104260008AE793E060E070E040EC50E00E946A3B37
:1042700008C08AE793E060E070E040EC50E00E9404
:10428000523BFF240DC00E94A332FBCF8FEF9FEF64
:1042900090936803809367036EDC84E793E0BEDC51
:1042A00083E793E06EEF7FEF0E949C2C45CF9BB994
:1042B0004498449A8BB94498449A0895459890E05C
:1042C000F6DF459A08950F931F93CF93DF93EC0188
:1042D0008B0160E070E020E030E0CB01BA01A90181
:1042E00098010E942B3C9B01AC0161157105810571
:1042F000910569F1E62FBB27A52F942F832F682FF7
:10430000CA01AA27BB27782F21116F5F61117F5F38
:104310002D2F3327CE0190702817390761F4CBB9C0
:104320004498449A4498449AE150D1F76150C1F7B7
:104330007150B1F70CC02BB94498449ACBB944984A
:10434000449AE150C1F76150B1F77150A1F7DF9184
:10435000CF911F910F9108950F931F938B01AEDFA3
:10436000C801A5DF1F910F910895CF93DF93DC0162
:10437000CD91DC911197FE018191282F332727FDE4
:1043800030951196FC93EE9327FF2FC025FF17C0A1
:10439000322F22273295307F8981482F552747FDBC
:1043A00050954F73507086E0440F551F8A95E1F782
:1043B000422B532B31961196FC93EE9308C0A90122
:1043C00076E0440F551F7A95E1F7407C5770ED91E8
:1043D000FC9111978191282F332727FD30952F735A
:1043E0003070242B352BED93FC93C901DF91CF91D5
:1043F0000895DC01ED91FC911197AF014F5F5F4F84
:1044000011965C934E93E4912E2F30E0E7FF31C07C
:10441000E5FF19C0322F22273295307F4F5F5F4F63
:1044200011965C934E9341505040FA018491482F6D
:1044300050E04F73507066E0440F551F6A95E1F7E6
:10444000422B532B08C0A90126E0440F551F2A9583
:10445000E1F7407C5770ED91FC9111973196ED9307
:10446000FC933197E4912E2F30E02F733070242B82
:10447000352BC9010895FF920F931F938A01F22EE5
:1044800080E2822769DF81E28F25B80165DF82E261
:1044900015DF1F910F91FF900895FF920F931F93C7
:1044A000CF93DF93EC01162F0CA1017067FF21C0A1
:1044B000002361F0862F90E09C01220F331F2470AF
:1044C000959587958270282B197F122B612F70E0AC
:1044D00067707070802F90E068277927E3E0660F9F
:1044E000771FEA95E1F780E390E16827792783E079
:1044F00033DFF12E16FF18C0102F110F6C857D854C
:1045000080E5812729DF6E857F8582E5812724DF8D
:104510006889798981E581271FDF6A897B8983E53D
:1045200081271ADF012F0695F4FE09C06881798181
:104530004A815B8120E0011121E0CE019CDFDF9107
:10454000CF911F910F91FF900895EF92FF920F93DB
:104550001F93CF93DF93FC01EA0104A1102F16955E
:1045600016951695212F30E086899789A489B589FB
:10457000A9014270507010FF1EC07B01E81AF90AB1
:10458000BE016A1B7B0BDB01452B29F06289738915
:104590006E0D7F1D04C0668577856E197F0922FF29
:1045A00005C0408951894A0F5B1F20C0448555854D
:1045B0004A1B5B0B1BC07B01EA1AFB0AC81BD90B09
:1045C000452B29F0608971896E0D7F1D04C06485BB
:1045D00075856E197F0922FF05C0428953894C0FEA
:1045E0005D1F04C0468557854C1B5D0B212F30E0B5
:1045F000802F90E02827392721703070CF013BDFD2
:10460000DF91CF911F910F91FF90EF900895FC01E2
:1046100084A186FF0FC02681378187FF07C0828172
:104620009381880F991F821B930B01C0C90193834B
:10463000828308952481358187FF07C0808191811D
:10464000880F991F821B930B01C0C901918380833E
:1046500008950F931F93CF93DF93FC01E901A5A168
:10466000A4FF0EC020853185620F731F828593855C
:10467000480F591FC20FD31F080F191FAF7EA5A3E4
:1046800084A180FD24C020E431E080EF90E077FF3A
:1046900002C060E070E0718F608F57FF02C040E0A1
:1046A00050E0538F428F0197C817D9070CF4CE0101
:1046B000958F848FC9010197081719070CF4C80159
:1046C000978F868FDF91CF911F910F91089520EFE3
:1046D00030E080E491E0DBCFFC01208D318D8485DA
:1046E0009585A901481B590B11A210A21416150695
:1046F00024F43587248751A340A3248D358D8089E8
:1047000091892817390714F4318B208B808991897E
:10471000019624853585821B930B958B848B20E035
:10472000181619060CF421E0822F0895FC0120814F
:104730003181808D918D28173907A4F0848D958D56
:10474000821793077CF042815381828D938D4817A5
:10475000590744F020E0868D978D841795071CF04B
:1047600021E001C020E0822F0895CF93DF93EC0178
:10477000DDDF882331F0CE0160E38FDE8FA198A5C5
:1047800096DDDF91CF910895FC0125A124FF0FC094
:1047900080819181860F971F91838083828193818D
:1047A000840F951F938382832F7E25A30895808590
:1047B0009185860F971F9183808382859385840FCF
:1047C000951F9383828308950F931F938C01DCDFE1
:1047D000C801CBDF1F910F910895FC0125A124FF93
:1047E0000FC080819181860F971F9583848382817A
:1047F0009381840F951F978386832F7E25A3089529
:1048000080859185860F971F958384838285938504
:10481000840F951F978386830895FC012481358139
:1048200080819181A901481B590B57FF0DC0358725
:10483000248788279927841B950B958B848B21507F
:104840003040280F391F09C095878487558B448BCA
:104850009C0121503040240F351F318B208B08954F
:104860000F931F938C01D9DFC8010296D6DF1F91E9
:104870000F910895CF92DF92EF92FF920F931F93C3
:104880007C01690181DFF70185A1806185A3C701F2
:10489000B601A801A2DFC701E3DF1F910F91FF90CE
:1048A000EF90DF90CF900895FC01808D918D9587DA
:1048B0008487828D938D97878687848D958D918B44
:1048C000808B868D978D938B828BCF0160ECE5CDAD
:1048D0002F923F925F926F927F928F929F92AF92B0
:1048E000BF92CF92DF92EF92FF920F931F93CF93DD
:1048F000DF93EC017B015A018901EEDE882309F484
:10490000AFC0CE010296E8DE882309F4A9C028A131
:1049100039A14AA15BA18CA1682F70E0DB01A870CE
:10492000B07083FF03C0CA01A9019C01F901E00F27
:10493000F11F4A9DC0014B9D900D5A9D900D112471
:10494000E80FF91F8C889D88CE88DF88AB2B19F083
:10495000C60164014C018F01B3E015950795BA9526
:10496000E1F70E0D1F1DA7E0EA2EF12CEE22FF222B
:104970001501281839084398F3E075956795FA955D
:10498000E1F76770606FCE0188DD6624F80144911D
:104990009701209530952770307081E090E002C03B
:1049A000880F991F2A95E2F7782E542E54018DA175
:1049B000272D30E0452D50E081FF12C02423352300
:1049C000232B19F46624639415C0662021F0CE01D0
:1049D000B501A601BADD8FA198A569DC66240AC0DD
:1049E00024233523232B19F08FA198A502C089A574
:1049F0009AA55DDC0894E11CF11C0894A108B1089B
:104A0000A114B10499F0872D90E095958795782EA3
:104A1000882369F60F5F1F4FF801849128EF3FEF5D
:104A2000E20EF31E582E70E8772EC1CF0894C1080D
:104A3000D108C114D10489F09701220D331DC90199
:104A400063E0959587956A95E1F7080F191F57E080
:104A5000E52EF12CE222F32299CFCE0125DF439AF5
:104A6000CE01D5DDDF91CF911F910F91FF90EF9097
:104A7000DF90CF90BF90AF909F908F907F906F907E
:104A80005F903F902F900895EF92FF920F931F93A6
:104A9000CF93DF93EC016CA31DA21EA260E070EE29
:104AA00040E050EE20E030E200E010E2D2DD198676
:104AB00018861B861A8688B1886388B987B188638F
:104AC00087B98FEF8AB9439806EF11E039C0F80132
:104AD0009491319625913491903611F1913618F4D4
:104AE000913029F406C09E3FC1F09F3F69F0B901A3
:104AF00023C08CA1682F70E07695762F6627779576
:104B000067956070717016C080ED97E0E0E9F1E0A4
:104B10003197F1F70197D1F711C0CE01C5DE0EC074
:104B20008CA1F82EF294FF0C80EEF822EE24B7014F
:104B300060707078622B732B892F0EDC0D5F1F4F16
:104B4000F2E00F351F0709F0C2CF439A18A61FA243
:104B50008FEF9FEF9AA789A78DA18D7F8DA3DF91FE
:104B6000CF911F910F91FF90EF9008954398FDDD35
:104B7000439A08950F931F938C0106DEC801F6DF58
:104B80001F910F9108952F923F924F925F926F92D3
:104B90007F928F929F92AF92BF92CF92DF92EF92CD
:104BA000FF920F931F93DF93CF93CDB7DEB7269776
:104BB000DEBFCDBF9E838D832B013A01890161E069
:104BC000262E312C221A330AC901880F991F222759
:104BD0003327281B390B3A8329834398ED81FE81C3
:104BE00085A18F7E85A3A801460D571D8D819E81CD
:104BF000B201EADDA301401B510B8D819E81B20100
:104C0000E3DDB801640D751D8D819E81A301DCDD9E
:104C1000B201601B710B8D819E81A301D5DD48011E
:104C200021E030E03C832B83AA24BB2456C037FC10
:104C30000AC008948108910889819A8102969A8312
:104C40008983280E391E0894A11CB11CEB81FC81BC
:104C50003296FC83EB832E0E3F1E6501C40CD51CDF
:104C60008401060D171D8D819E81B601A801ACDD62
:104C70007201EA18FB088D819E81B701A801A4DDAD
:104C80008301081919098D819E81B601A8019CDD57
:104C90008D819E81B701A80197DD6401C40CD51CEC
:104CA0008501060D171D8D819E81B601A8018CDD41
:104CB0007201E818F9088D819E81B701A80184DD91
:104CC00083010A191B098D819E81B601A8017CDD33
:104CD0008D819E81B701A80177DDA814B9040CF479
:104CE000A6CF439A2696DEBFCDBFCF91DF911F910D
:104CF0000F91FF90EF90DF90CF90BF90AF909F907B
:104D00008F907F906F905F904F903F902F9008957D
:104D1000CF93DF93EC01E0DC882399F0CE0102967B
:104D2000DBDC882371F04398CE0160EFB6DB6C8941
:104D30007D894E895F898FA198A5C5DACE01B4DD42
:104D4000439ADF91CF9108952F923F924F925F92B5
:104D50006F927F928F929F92AF92BF92CF92DF928B
:104D6000EF92FF920F931F93DF93CF9300D000D069
:104D7000CDB7DEB72C013B015A0149011C830B83DF
:104D80002617370714F44B0139018B819C818A1552
:104D90009B052CF48B819C81BC82AB825C0114014D
:104DA0002618370894E02916310408F466C0EB8110
:104DB000FC81EA19FB09FA83E983349708F45DC0A2
:104DC00063010894C11CD11C85010F5F1F4FC201F4
:104DD000B601A801CFDEAEEFEA2EAFEFFA2EE80C57
:104DE000F91CC201B701A801C5DE0B811C8102506C
:104DF0001040C201B601A801BDDEC201B701A80181
:104E0000B9DEF2E0EF2EF12CE60CF71CECEFCE2E23
:104E1000EFEFDE2EC20CD31CC201B701A501960133
:104E200001E010E00E94F71B8B819C8101979C831D
:104E30008B83C201B7014B815C8196010E94F71BF5
:104E400072E0E72EF12CEA0CFB1CC980DA80ECEF53
:104E5000FFEFCE0EDF1EC201B301A70121E030E05B
:104E600086010E94F71B089481089108C201B401D1
:104E7000A70121E030E00E94F71B2496DEBFCDBFE2
:104E8000CF91DF911F910F91FF90EF90DF90CF9026
:104E9000BF90AF909F908F907F906F905F904F905A
:104EA0003F902F900895EF92FF920F931F937C01F4
:104EB000C901F801D70195960C9110E001701070AE
:104EC0009801261B370B280F391F041B150B0E0FDB
:104ED0001F1FC701CFDCC7011BDF1F910F91FF9080
:104EE000EF9008952F923F924F925F926F927F9230
:104EF0008F929F92AF92BF92CF92DF92EF92FF92EA
:104F00000F931F93DF93CF9300D000D0CDB7DEB7C0
:104F10001C013B015C834B8359014801FA82E98201
:104F20002617370714F45B0139018B819C818816A1
:104F300099062CF4C4018B809C809C838B83F101A7
:104F400085A18F7E85A3E980FA80E60CF71C898114
:104F50009A818E0D9F1D8A159B056CF449805A809D
:104F60008B819C81480E591E89819A81840D951DE3
:104F7000881599053CF0C101B3014B815C81950115
:104F8000840122C06401E981FA81CE1ADF0AC101DD
:104F9000B3014B815C819701860185DFC101B701B7
:104FA0004B815C81950182017EDF750189819A8147
:104FB000E81AF90AC101B701A2019501840173DF62
:104FC000C101B301A60197016EDF2496DEBFCDBFFC
:104FD000CF91DF911F910F91FF90EF90DF90CF90D5
:104FE000BF90AF909F908F907F906F905F904F9009
:104FF0003F902F900895CF92DF92EF92FF920F9300
:105000001F93CF93DF93EC01E8DBCE0129DC6C89A1
:105010007D896115710579F48C859D85998B888BC7
:105020002DA130E0217030708A899B89820F931FF7
:105030009B8B8A8B13C04E895F8941155105C9F43A
:105040008E859F859B8B8A8B2DA130E021703070DF
:1050500088899989820F931F998B888BCE0158DE9E
:105060008C819D81998388838E819F819B838A8394
:1050700057C02C813D81888199812817390724F0F8
:1050800001E0C02ED12C03C0CC24CA94DC2C2E818C
:105090003F818A819B812817390724F011E0E12E96
:1050A000F12C03C0EE24EA94FE2C8B01041B150B9B
:1050B000439822C0CE0159DBA801440F551F2E8909
:1050C0003F89CA01820F931F1816190644F4021B68
:1050D000130B888199818C0D9D1D998388838C8900
:1050E0009D894817590744F4080F191F8A819B812D
:1050F0008E0D9F1D9B838A83288139818C819D81A0
:1051000028173907B9F62A813B818E819F8128179C
:10511000390781F68DA180FF02C0CE0126DB439ABC
:10512000DF91CF911F910F91FF90EF90DF90CF9083
:1051300008952F923F924F925F926F927F928F923B
:105140009F92AF92BF92CF92DF92EF92FF920F9316
:105150001F93DF93CF93CDB7DEB72697DEBFCDBFCA
:105160009C838B832B015E834D83A9013801261715
:10517000370714F4AB0129018D819E8168167906E9
:105180002CF4C3016D807E809E838D83FA01E41927
:10519000F509FA83E983E430F10508F45EC01301F0
:1051A0008D819E81281A390A94E02916310408F469
:1051B00054C092E0A92EB12CA40CB51C4F01ECEF09
:1051C000FFEF8E0E9F1E8B819C81B5014D815E810C
:1051D000940101E010E00E94F71B72010894E11CA9
:1051E000F11CC980DA808EEF9FEFC80ED91EED81C9
:1051F000FE813196FE83ED838B819C81B701AF01E7
:1052000096010E94F71B8D819E8101969E838D835E
:10521000ECEFFFEF2E0E3F1E8B819C81B2014D8182
:105220005E8129813A8181010E94F71B8EEF9FEFF9
:10523000680E791E8B819C81B701A301960101E064
:1052400010E00E94F71B0894611C711C8B819C81EB
:10525000B501A30194010E94F71B2696DEBFCDBFC6
:10526000CF91DF911F910F91FF90EF90DF90CF9042
:10527000BF90AF909F908F907F906F905F904F9076
:105280003F902F9008952F923F924F925F926F928E
:105290007F928F929F92AF92BF92CF92DF92EF92C6
:1052A000FF920F931F93DF93CF9300D000D0CDB721
:1052B000DEB73C017A836983FC0185A18F7E85A3DB
:1052C000AA24BB24A21AB30A229F1001239F300CE8
:1052D000329F300C11242501440E551E4A018A18B4
:1052E0009B08BC82AB8235C0229FC001239F900DDA
:1052F000329F900D1124840F951F28163906CCF08B
:10530000E980FA80E20EF31E220F331FCC24DD2445
:10531000C21AD30AC301B701A201960101E010E04D
:105320000E94F71BC301B701A40196010E94F71B5D
:1053300005C02F5F3F4F12161306B4F68B819C8178
:1053400001969C838B830894411C511C089481080E
:105350009108EB81FC811E161F064CF0EE9FA00108
:10536000EF9F500DFE9F500D11249501E4CF249620
:10537000DEBFCDBFCF91DF911F910F91FF90EF90D6
:10538000DF90CF90BF90AF909F908F907F906F9065
:105390005F904F903F902F900895EF92FF920F9360
:1053A0001F938C017B0143987FDAC80160EF75D8A9
:1053B000C70160EF70E040E451E00E946321439A2E
:1053C0001F910F91FF90EF9008959C0181389105F6
:1053D0009CF084EB91E0FC014591549142175307F6
:1053E00021F0452B49F00296F6CF009729F09C0159
:1053F000245B304035952795C90108957F928F929F
:105400009F92AF92BF92CF92DF92EF92FF920F9353
:105410001F93CF93DF938C01FC0185A182FF43C0D2
:105420006A30710509F03FC084A1982F9695969532
:1054300096959827892F8295869586708927482F7B
:1054400080FF18C0828593859383828386A52081FF
:10545000318141FF06C0992787FD9095281B390BA4
:1054600006C0992787FD9095280F391FF8013183D1
:105470002083D2C0F801808591859183808386A5A1
:105480002281338142FF06C0992787FD9095281B12
:10549000390B06C0992787FD9095280F391FF80111
:1054A00033832283B9C0CB0190DF9C01F80147A56B
:1054B00050A9841795073CF081A992A9840F951FE4
:1054C0002817390714F02FE330E04901841A950AB0
:1054D000F80165A576A4E3A4F4A416160CF455C04F
:1054E000A1A8B2A8603FD9F4C0E0D0E0CC24DD246C
:1054F00080E020E030E00EC0F701949128153905D6
:1055000011F4892F6E010894E11CF11CC90FD11D03
:105510002F5F3F4F2A153B057CF3682F5DC0C0E02D
:10552000D0E0CC24DD2430E042E050E0A1E0B0E067
:10553000F7010894E11CF11C7491272F2F70261B92
:10554000CA0102978815990511F4322F6E01C20F16
:10555000D11DAA15BB0599F0872F90E0E4E0959541
:105560008795EA95E1F78F70861BA815B90511F4A8
:10557000382F6E01C80FD11D4A155B0511F4632F3A
:105580002BC04E5F5F4F1296D3CFC62FDD27C7FDCE
:10559000D0952796C87F8C2F90E073E095958795DE
:1055A0007A95E1F7272D332727FD3095A901849FB0
:1055B0009001859F300D949F300D1124882D90E02F
:1055C000FC012E9FC0012F9F900D3E9F900D112436
:1055D000E80EF91ECC24DD24F80184A1982F83FF66
:1055E00003C0872D762E682F94FD619595FD7194EB
:1055F000F80185A1806185A3772767FD7095472D08
:10560000552747FD5095C801E8D8C80129D9C801D8
:10561000B701AE0196015CD9DF91CF911F910F9137
:10562000FF90EF90DF90CF90BF90AF909F908F90C2
:105630007F900895FC0186A1282F30E0C9018F706A
:105640009070892B01F121FF02C07595679584A1A7
:1056500083FF0CC02281338185FF03C0260F371FD3
:1056600002C0261B370B33832283089520813181AA
:1056700084FF05C0260F371F318320830895261B22
:10568000370B318320830895DC01FB019D968C91BB
:105690009D97482F552747FD509514161506ACF1D8
:1056A0009F966D917C91D097E617F70754F09F0174
:1056B000260F371FD1968D919C91D29728173907C5
:1056C00014F0EFE3F0E09F01261B370B9B96ED9162
:1056D000FC919C978FEF403F580731F4E20FF31F86
:1056E0008491482F50E011C0C90195958795E80F26
:1056F000F91F849120FF02C082958F7090E08F7017
:1057000090709C01241B350BA901CA010895EF92EA
:10571000FF920F931F93DF93CF9300D0CDB7DEB7E7
:105720007C017A83698300E010E0CE0101960E943B
:10573000B521BC01009729F0C701A6DF080F191F8A
:10574000F4CFC8010F900F90CF91DF911F910F916F
:10575000FF90EF9008950F931F93DF93CF9300D0A6
:10576000CDB7DEB78C017A836983FC0186A190E016
:105770008F709070892B19F460E070E005C069812A
:105780007A81C801C4DFBC01C80154DFCE01019693
:105790000E94B521BC01009719F0C8012FDEF6CF99
:1057A0000F900F90CF91DF911F910F910895EF927D
:1057B000FF920F931F93DF93CF9300D0CDB7DEB747
:1057C0007C017A83698300E010E0CE0101960E949B
:1057D000F921BC01009729F0C70156DF080F191FF6
:1057E000F4CFC8010F900F90CF91DF911F910F91CF
:1057F000FF90EF9008950F931F93DF93CF9300D006
:10580000CDB7DEB78C017A836983FC0186A190E075
:105810008F709070892B19F460E070E005C0698189
:105820007A81C801C4DFBC01C80104DFCE01019642
:105830000E94F921BC01009719F0C801DFDDF6CF05
:105840000F900F90CF91DF911F910F910895DC0180
:10585000FB01CB010196E4919D96EC939D979C01F1
:105860002F5F3F4FFC0184919E968C939E97C901B8
:105870000196F90124919F962C939F97D0961C92A4
:10588000D097FC012491D1962C93D197D2961C925B
:10589000D29701969C969C938E939B97089518950A
:1058A000282F30E027FF02C0409A01C0409881E0D5
:1058B000982F9A95F1F7419A982F9A95F1F7220F20
:1058C00041988A95F1F718992F5F3F5F383051F76B
:1058D000822F0895EBE6F0E080818260808388B1BA
:1058E0008C7F88B987B1836087B985B1836085B9BA
:1058F00080E0D6DF80E0D4DF80E0D2CF83B1869530
:105900008095817008951F93862FCADF88E08A955D
:10591000F1F780E0C5DF182F80E0C2DF512F40E0B3
:10592000282F30E0242B352B86E0369527958A9555
:10593000E1F7C9011F910895199B0CC081E08BBB51
:1059400090916800809168008160809368008895DC
:105950009093680080E008956F927F928F929F925B
:10596000AF92BF92CF92DF92EF92FF920F931F936D
:105970003B015A0149017801E21AF30A0027F7FCBA
:105980000095102F9C01261B370B442737FD4095AF
:10599000542FC801B7010E942B3CA618B708CC248D
:1059A000B7FCC094DC2CA60195010E94763C820EC7
:1059B000931EC4011F910F91FF90EF90DF90CF9045
:1059C000BF90AF909F908F907F906F900895FF92BF
:1059D0000F931F93609164036170606D83E793E0A0
:1059E00092DF60913A0470913B0440913E045091E3
:1059F0003F04F0906403F0FC03C000EF10E002C02D
:105A000000E411E020E030E0A7DF909343048093AE
:105A1000420481E0F82280E9F82A83E793E06F2DC1
:105A200072DF9C0160913C0470913D044091400400
:105A3000509141048091640380FD03C000E411E0B3
:105A400002C000EF10E0C90120E030E085DF909354
:105A50004504809344041F910F91FF900895909105
:105A60006403492F50E09A0135952795822780FDE0
:105A700003C064E170E009C040FD03C060EF70E066
:105A800002C060E471E06451704081FD03C044E1F4
:105A900050E009C040FD03C040E451E002C040EFC7
:105AA00050E04451504080E493E024E130E0EBCBFF
:105AB000CF93DF93EC0183E793E020DF882359F451
:105AC000219751F088EE93E0E0E9F1E03197F1F7AA
:105AD0000197D1F7F0CF81E0DF91CF910895CF9278
:105AE000DF92EF92FF920F931F93CF93DF9380E4A7
:105AF00093E060E070EE40E050EE20E030E200E045
:105B000010E20E9429238AE290E06AE270E00E949B
:105B1000181C8091640390E09C012170307080FD1E
:105B200003C060EF70E002C060E471E0EB01D59566
:105B3000C795232B19F440E451E002C040EF50E038
:105B40007A01F594E79480E493E0BE0140E050E0F0
:105B50000E94C42380E493E060E775E34CDE40914B
:105B60006E03552747FD509580E493E0BE010E94E7
:105B7000C42380E493E064E675E33DDE89E59EECB2
:105B8000909368038093670380E493E062E070E0A1
:105B90004AE250E00E94C4238091650380618093B3
:105BA000650380E493E06CEE70E04CEE50E00E9400
:105BB000ED2380E493E00E940D2482E493E00E94B0
:105BC0000D2480E493E0A4D880E098EF90936803DC
:105BD0008093670310E0812F42DF1F5F1430D9F7F5
:105BE00080E493E06CE775E132DE82E08093660347
:105BF0008FE190E0909368038093670389E59EECC2
:105C000090936A0380936903809165038D7F8093ED
:105C1000650380916E03992787FD9095A701481B26
:105C2000590B80E493E0BE010E94C42380E493E01A
:105C30006DE475E3E0DD80E493E0BE01A7010E941E
:105C4000C42380E493E068E375E3D5DD80EE97E05C
:105C50009093680380936703FF248CE291E028DF30
:105C6000882309F4E3C0609164036170606D83E789
:105C700093E049DE8C01609164036170606983E7A1
:105C800093E041DE21E00038120714F460E006C022
:105C900022E0003812070CF4C9C061E0AC0181E0D9
:105CA0004038580734F022E0403852070CF4BEC0A8
:105CB0006260262F30E0F901EE0FFF1FEE0FFF1F8D
:105CC000EA5BFB4F11830083F901EE0FFF1FEE0F1C
:105CD000FF1FE85BFB4F5183408381E090E0062E7D
:105CE00002C0880F991F0A94E2F7182F90E02F2D19
:105CF00030E082239323892B19F4862FB0DEF12A1A
:105D000088EE93E0E0E9F1E03197F1F70197D1F700
:105D10008FE0F81609F0A1CF00914E0410914F04C6
:105D20008091460490914704080F191F1595079517
:105D3000E0905204F090530480914A0490914B04F7
:105D4000E80EF91EF594E7948091640390E041E039
:105D5000C42ED12CC822D92280FD03C0C0EFD0E0D0
:105D600002C0C0E4D1E0B701601B710B882777FD4A
:105D70008095982F24E130E040E050E00E942B3CD9
:105D8000A8979E01442737FD4095542F0E94763CEA
:105D9000021B130B10933B0400933A042E0D3F1D7E
:105DA00030933F0420933E0400914C0410914D0425
:105DB0008091480490914904080F191F1595079583
:105DC000E0905404F0905504809150049091510457
:105DD000E80EF91EF594E794CD2819F4C0E4D1E05B
:105DE00002C0C0EFD0E0B701601B710B882777FDC0
:105DF0008095982F24E130E040E050E00E942B3C59
:105E0000A8979E01442737FD4095542F0E94763C69
:105E1000021B130B10933D0400933C042E0D3F1DF9
:105E2000309341042093400481E001C080E0DF9181
:105E3000CF911F910F91FF90EF90DF90CF90089539
:105E4000FC0181816281833024F4A82FA65F615018
:105E500002C0A82FA250772767FD70954381552770
:105E600047FD50952081332727FD3095225F3F4F16
:105E7000CA019595879595958795280F391F440FE9
:105E8000551F241B350B260F371F75956795759584
:105E90006795260F371F83EFA802C0011124809554
:105EA000909565E070E00E94633CC901860F971FE2
:105EB00067E070E00C94633CFC012181223061F4C6
:105EC0008281992787FD909583709070892B11F4BA
:105ED0008DE108958CE10895332727FD3095C901A0
:105EE000F3E095958795FA95E1F78227932780FD52
:105EF00002C08EE108958FE10895FC0181818F5FDA
:105F000081838D302CF081E0818382818F5F828359
:105F100008951F93CF93DF93EC0118811F5F1883BF
:105F2000CBDF811724F481E08883CE01E6DFDF91A7
:105F3000CF911F910895FC01818181508183882335
:105F400029F48281815082838CE081830895CF93EC
:105F5000DF93EC01888181508883882329F4CE0166
:105F6000EADFCE01A9DF8883DF91CF910895FC019C
:105F7000908180911601981791F491818091170179
:105F8000981769F4928180911801981741F420E0E4
:105F9000938180911901981719F421E001C020E044
:105FA000822F0895A0915604B09157046091420445
:105FB000709143044091440450914504EFE5F4E0AE
:105FC00020E030E017C080819181681779077CF06C
:105FD000848195816817790754F4828193814817E9
:105FE00059072CF0868197814817590744F02F5F95
:105FF0003F4F38962A173B0734F32FEF3FEFC90185
:1060000008951092130185E38093140192E0909318
:10601000150183E0809316019093170181E180932D
:10602000180108950F931F9360E070EE40E050EE6A
:1060300020E030E200E010E20E9429231F910F913E
:106040000895EF92FF920F931F938C017B01BA0189
:10605000A9010E94C423C801B701CDDB1F910F9194
:10606000FF90EF9008952F923F924F925F926F9220
:106070007F928F929F92AF92BF92CF92DF92EF92D8
:10608000FF920F931F93DF93CF93CDB7DEB72E9779
:10609000DEBFCDBF2C017E876D8758874F831A875F
:1060A0000987FC86EB8637FF05C080E493E0BA01E0
:1060B0002EDB9C0186EF9FEF480E591EC901959576
:1060C00087957201E81AF90AAAE0B0E04A0E5B1E51
:1060D00044E1C42ED12CC20ED31ECE0CDF1C2EEFF9
:1060E000A22E2FEFB22EED85FE85AE0EBF1E99E1DA
:1060F000892E912C8E0E9F1E88E1682E86EC782EBC
:10610000709268036092670380E493E0B701A50191
:10611000960184010E94532729853A8530936803AC
:1061200020936703C70102979E838D83D501129741
:10613000BC83AB830BE1202E312CED85FE852E0E2A
:106140003F1E80E493E06D817E81AD019701810166
:106150000E94532796012E5F3F4F3A83298380E4A4
:1061600093E0B7014B815C8185010E9453278B85A9
:106170009C85909368038093670380E493E0B60165
:10618000A50129813A8181010E94532780E493E08F
:10619000B701A40196010E9453270894E108F10871
:1061A0004D855E85465E5F4F80E493E0B7010E94B7
:1061B000C42380E493E00E94B6250894C11CD11C3E
:1061C0004D855E854350504080E493E0B6010E94C7
:1061D000C42380E493E00E94B62580E493E0B201FA
:1061E0004D855E850E94C423109268031092670358
:1061F00070926A0360926903809165038D7F80933A
:10620000650380E493E06F817885A5DAA985BA8576
:10621000EB85FC85AE17BF0741F1E0915604F09184
:1062200057043196F0935704E0935604319713E0E6
:10623000EE0FFF1F1A95E1F7CF01815A9B4F2D8179
:106240003E81DC012D933C93AF014F595B4F2B8175
:106250003C81DA012D933C93ED59FB4FA981BA8122
:10626000B183A083FC01378226822E96DEBFCDBF8C
:10627000CF91DF911F910F91FF90EF90DF90CF9022
:10628000BF90AF909F908F907F906F905F904F9056
:106290003F902F900895CF92DF92EF92FF920F934D
:1062A0001F93C0904203D090430320914A03309142
:1062B0004B03C21AD30A00D000D000D0EDB7FEB70E
:1062C00031960FEC14E0ADB7BEB712961C930E9347
:1062D00011972FEA35E33383228395838483F3D7A1
:1062E0008DB79EB706969EBF8DBF8CE890E0B60135
:1062F000A80120E530E00FE110E0FFE1EF2EF12CE6
:10630000B2DE8CE390E0B60140E051E02FEF3FEFCA
:106310000EE917EFE0E1EE2EE4E8FE2EA4DE8CEDB0
:1063200090E0B60144E051E02FEF3FEF9CDE1F917B
:106330000F91FF90EF90DF90CF900895DF92EF9252
:10634000FF920F931F93D82E87FF6CC083E190E0DC
:1063500062E070E00E94181C80E493E069E975E354
:1063600048E750E020E030E06CDEB9E5EB2EBEEC13
:10637000FB2EF0926803E092670380E493E062E012
:1063800070E043E150E02CEE30E00BE211E00E94BF
:106390003A2480E493E00E948826109268031092C9
:1063A0006703F0926A03E0926903809165038D7F31
:1063B000809365031092660380E493E064E975E3DB
:1063C00041E050E022E230E03CDE80E493E06FE820
:1063D00075E341E050E028E430E033DE80E493E010
:1063E0006BE875E341E050E02EE630E02ADE80E421
:1063F00093E066E875E341E050E024E930E021DE17
:1064000080E493E061E875E341E050E02AEB30E09E
:1064100018DE80E493E06CE775E341E050E020EEA5
:1064200030E00FDE80E493E06CE775E110DA82E0A3
:106430008093660380E493E068E770E04EE150E00B
:106440000E94C42310925704109256041D2DD0FEB2
:106450000EC080915E0424E68202C00111242091C6
:106460005D04332727FD3095820F931F14DF88E7E3
:1064700090E066E270E00E94921B11FF06C08091DE
:106480005C04992787FD909506DF88E790E066E237
:1064900070E00E94921B12FF06C080915B04992756
:1064A00087FD9095F8DE88E790E066E270E00E9454
:1064B000921B13FF06C080915A04992787FD90957F
:1064C000EADE88E790E066E270E00E94921B14FF2B
:1064D00006C080915904992787FD9095DCDE88E7F6
:1064E00090E066E270E00E94921B15FF06C080916A
:1064F0005804992787FD9095CEDE88E790E066E204
:1065000070E00E94921BD7FE18C088E290E064E021
:1065100071E046E051E02FEF3FEF0EE917EFA0E109
:10652000EA2EA4E8FA2E9FDD80EA90E064E071E0B4
:1065300049E051E02FEF3FEF96DD1F910F91FF9063
:10654000EF90DF900895CF92DF92EF92FF920F933A
:106550001F93CF93DF93A8E5B4E0E3E1F1E087E098
:1065600001900D928150E1F780E493E05BDD8FEFC5
:10657000E5DE109249031092480310924B031092EB
:106580004A0380E493E04EDD88E592E091DA8823C7
:1065900009F47AC180EE9FEF9093680380936703BC
:1065A000CC24DD24EE24FF240FE311E0CFEED0E075
:1065B00078C00DDA80E89FEF9093680380936703BB
:1065C0006091420470914304409144045091450409
:1065D00080E493E024E130E00E9443298FE190E0E1
:1065E0009093680380936703609142047091430421
:1065F000409144045091450480E493E024E130E06C
:106600000E94C32560914204709143044091440468
:106610005091450480E493E025E130E00E94C325D9
:1066200060914204709143044091440450914504A8
:1066300080E493E026E130E00E94C32540914204CB
:1066400050914304CA014597C817D90714F0EA01CD
:1066500066972091440430914504C9014597081775
:1066600019071CF0890106511040CA0145968E1584
:106670009F052CF096E1E92EF12CE40EF51EC901E0
:1066800045968C159D052CF086E1C82ED12CC20EA6
:10669000D31E80ED97E0E0E9F1E03197F1F7019743
:1066A000D1F783E793E02AD9882309F082CF80E4E9
:1066B00093E0BE01A801970186010E9429238FEF74
:1066C0003DDE80E493E0AEDC6DDCEC0186309105CC
:1066D00009F486C087309105BCF48230910509F435
:1066E0004EC0833091053CF4009759F181309105FB
:1066F00009F03FCF34C08430910509F456C085308D
:1067000091050CF05EC045C08A30910509F492C035
:106710008B3091054CF48830910509F476C08930AE
:1067200091050CF07DC067C08C30910509F497C0CD
:106730008C3091050CF489C08D30910509F019CF8A
:10674000A3C080915D04815080935D0487FF92C057
:1067500083E680935D0480915E0481500DC080913A
:106760005D048F5F80935D0484360CF483C01092C7
:106770005D0480915E048F5F80935E047BC0809196
:106780005C04815080935C0418160CF473C08CE098
:1067900009C080915C048F5F80935C048D300CF4A1
:1067A00069C081E080935C0465C080915B04815086
:1067B00080935B0418160CF45DC08BE594E07CDBE1
:1067C0000CC010915B041F5F10935B048BE594E099
:1067D00073DB81170CF04EC081E080935B044AC0EC
:1067E00080915A04815080935A0487FF43C087E107
:1067F00080935A043FC080915A048F5F80935A045B
:106800008831C4F110925A0435C0809159048150E6
:106810008093590487FF2EC08BE3809359042AC0CC
:10682000809159048F5F809359048C331CF110922E
:10683000590420C08091580481508093580487FFE8
:1068400019C08BE38093580415C0809158048F5F62
:10685000809358048C3374F0109258040BC0A3E159
:10686000B1E0E8E5F4E087E001900D928150E1F7B6
:1068700081E00BC0D595C79581E090E002C0880FFC
:10688000991FCA95E2F774CE80E0DF91CF911F91F6
:106890000F91FF90EF90DF90CF900895FC01418120
:1068A0004150440F440F462B8081815090E0440FAB
:1068B000440F9C0153E0359527955A95E1F7422BFB
:1068C000EAE7F3E0E40FF11D8770907021E030E01B
:1068D00002C0220F331F8A95E2F780818223089538
:1068E000FF920F931F93CF93DF93EC01FF2401E0FE
:1068F00010E0CE01612FD2DF8111F02A1F5F14302A
:1069000011F0000FF6CF8F2DDF91CF911F910F91D6
:10691000FF9008951F93CF93DF93EC01162F90DA29
:10692000E82F882309F44CC04881413039F489812B
:10693000813009F445C0853081F442C0433011F004
:106940004F3121F489818A3041F43AC0493111F044
:106950004A3119F489818C3099F15981252F2350BE
:10696000253030F58FE12802C0011124840F223038
:106970000CF081508823E1F0282F332727FD309534
:10698000612F772767FD7095CB010297281739078C
:10699000B9F0CB0101962817390791F0CB01879602
:1069A0002817390769F06E5C7F4F2617370741F0CB
:1069B000E33041F45B3031F480E04051473018F46B
:1069C00081E001C080E0DF91CF911F9108954F9247
:1069D0005F926F927F928F929F92AF92BF92CF926F
:1069E000DF92EF92FF920F931F93CF93DF934B01B0
:1069F000B42EF1EFCF2EFFEFDF2EC80ED91EEB0124
:106A0000219747FD03C089E59EEC02C080E098EF26
:106A10009093680380936703B60161507040AE01A4
:106A2000415050409601215E3F4F8E010B5E1F4F3B
:106A300080E493E0E1E0EE2EF12C0E94722780E8E2
:106A4000B81601F59601225E3F4F80E493E0B6014F
:106A5000AE0164968E010E94722789E59EEC9093A8
:106A60006803809367039601235E3F4F219780E47C
:106A700093E00894C11CD11CB601A4018E010E94B0
:106A800072278EC03FE0E32EEB2021F429E53EEC97
:106A9000FF2411C0EE2DF0E0E550FA4C4491842F14
:106AA00090E083709070880F991F86599F4FFC016A
:106AB00025913491F42E309368032093670382E08C
:106AC000A82EB12CAC0CBD1C02E1402E512C4C0E5A
:106AD0005D1E80E493E0B601AE01950182010E9443
:106AE0005327EE2081F0F694F694EF2DF0E0E3705A
:106AF000F070EE0FFF1FE659FF4F85919491909330
:106B0000680380936703BEE16B2E712C6C0C7D1CB7
:106B10008E010E5F1F4F80E493E0B501AE0193013B
:106B20000E945327EE2081F0F694F694EF2DF0E0CA
:106B3000E370F070EE0FFF1FE659FF4F85919491BF
:106B40009093680380936703ECE18E2E912C8C0C5C
:106B50009D1C74E1A72EB12CAC0EBD1E80E493E009
:106B6000B401AE01930185010E945327EE2081F00C
:106B7000F694F694EF2DF0E0E370F070EE0FFF1F47
:106B8000E659FF4F85919491909368038093670332
:106B900080E493E0B601A201940185010E9453278D
:106BA000DF91CF911F910F91FF90EF90DF90CF90E9
:106BB000BF90AF909F908F907F906F905F904F901D
:106BC00008958F929F92AF92BF92CF92DF92EF92F1
:106BD000FF921F93CF93DF93EC015B014A01122FC9
:106BE000B9E0CB2ED12CC80ED91EA9E0EA2EF12C8B
:106BF000E60EF71E80E493E0B601A70129E030E03D
:106C00000E94C325112341F080E493E0B601A7015F
:106C100025E030E00E944329669680E493E0BE01BF
:106C2000A5010E94C42380E493E0B4010E94FB2BE1
:106C3000DF91CF911F91FF90EF90DF90CF90BF90A9
:106C4000AF909F908F9008952F923F924F925F92B6
:106C50006F927F928F929F92AF92BF92CF92DF926C
:106C6000EF92FF920F931F93DF93CF93CDB7DEB7D1
:106C70002897DEBFCDBF8091160190911701A0919A
:106C80001801B091190189839A83AB83BC8380E496
:106C900093E060E070EE40E050EE20E030E200E093
:106CA00010E20E94292383E190E062E070E00E94FC
:106CB000181C80E493E068E770E040E050E00E9438
:106CC000C42380E493E06DEE75E30E94FB2B8824DF
:106CD0003324992401C0882419E5C12E1EECD12E3D
:106CE000D0926803C092670380E493E062E070E0B2
:106CF00043E150E02CEE30E00BE211E00E943A2438
:106D000080E493E00E948826109257041092560463
:106D10006A81772767FD7095615070408AE790E03F
:106D20000E943E1E2DB73EB7285030403EBF2DBFBB
:106D3000EDB7FEB7319605ED14E0ADB7BEB71296CC
:106D40001C930E93119723EE35E3338322839583AF
:106D500084838B81992787FD909597838683B3D20F
:106D60002DB73EB7285F3F4F3EBF2DBF88E790E06D
:106D70006EE170E0A80128E730E00FE110E0BFE12C
:106D8000EB2EF12C70D984E190E06EE170E04AE1E5
:106D900051E02FEF3FEF0EE917EFA0E1EA2EA4E854
:106DA000FA2E61D98CED90E06EE170E04CE151E09B
:106DB0002FEF3FEF58D9882009F447C082EC90E0CC
:106DC0006AEF70E04EE151E02FEF3FEF4CD91092A7
:106DD0006603D0926A03C0926903809165038D7F38
:106DE0008093650320E0992009F421E08AE090E097
:106DF00065EF70E04EED55E3E4DE20E031E0931600
:106E000009F421E08AE090E063E171E049ED55E3A7
:106E1000D8DE20E082E0981609F421E080E590E0D9
:106E200065EF70E044ED55E3CCDE20E093E0991689
:106E300009F421E080E590E063E171E04EEC55E378
:106E4000C0DE82E08093660323C082E390E06AEFB5
:106E500070E046E251E02FEF3FEF0EE917EFF0E16F
:106E6000EF2EF4E8FF2EFFD8332019F44EE251E064
:106E700002C046E351E084EB90E06AEF70E02FEF50
:106E80003FEF0EE917EFE0E1EE2EE4E8FE2EEBD83F
:106E90008FE190E0909368038093670389E59EEC0F
:106EA00090936A0380936903809165038D7F80933B
:106EB0006503DD24D39438E1E32EF12C6D2D772783
:106EC00067FD709582EB95E30E943E1E00D000D0D6
:106ED00000D0EDB7FEB7319605ED14E0ADB7BEB703
:106EE00012961C930E9311972BEC35E33383228378
:106EF00095838483E8D12DB73EB72A5F3F4F3EBFCD
:106F00002DBF80E493E0B7014CE350E00E94C4231E
:106F100080E493E0B8010E94AB2BD39437E0D31602
:106F200009F4DD2480E290E0E80EF91E98EFE916FE
:106F3000F10421F6109268031092670380E493E055
:106F400068E070E040E550E028EE30E001E510E058
:106F50000E9453273B81832F8B5F63E19BD4492F92
:106F600083E19802C0011124885E6EE193D4292F39
:106F7000842F6BE09BD4820F6DE18CD42B5E281B99
:106F8000832F859585953E5F830F67E083D4892F96
:106F9000820F87507FD4295FB22EB91A89819A81D6
:106FA000AB81BC818D839E83AF83B88781E08D8365
:106FB000CE0105960E94202F182F82300CF4195F05
:106FC000CE0105960E94A72F11501130C9F74D80B0
:106FD0005E806F80788481E090E0092C02C0880F89
:106FE000991F0A94E2F7282E28E5C22ED12C70C0F2
:106FF0003E812A81321719F080E194E802C080E0D6
:1070000090E09093680380936703321761F4CE0198
:1070100005966B2D7FDC882331F080E098EF90930C
:1070200068038093670300D000D000D0EDB7FEB7AF
:10703000319605ED14E0ADB7BEB712961C930E93D2
:10704000119788EC95E3938382838D81992787FD3F
:1070500090959583848337D12DB73EB72A5F3F4FF4
:107060003EBF2DBF80E493E0B701A6010E94C42378
:1070700080E493E0B8010E94AB2B9E818A8198172F
:1070800091F4CE0105962CDC182F81101221CE012F
:1070900005960E94B72F81111068112321F0C701B6
:1070A000B601412F94DCCE0105960E94892F80E223
:1070B00090E0E80EF91E98EFE916F10409F098CF78
:1070C000A8E1B0E0CA0EDB1EB8EECB16D10461F029
:1070D00098E1E92EF12C8CCF88EE93E0E0E9F1E025
:1070E0003197F1F70197D1F783E793E00E947E2C67
:1070F000882391F788E592E00E94582D882309F4AF
:10710000BFC00E94E72C0E94D22F8130910589F0E8
:10711000823091051CF4892B39F013C0823091051F
:1071200069F0039771F4ADC0CE0101960E949B2FC8
:10713000D3CDCE0101960E947D2FCECD81E0882651
:10714000CBCD882089F22091440430914504C901B7
:10715000805F9040CC9788F499242E50314014F0F1
:107160009924939480914204909143048035910531
:107170000CF4B2CD92E0992AAFCD4D825E826F823F
:10718000788688E5A82EB12C77C0209142043091F2
:107190004304C6014097281739070CF457C0C601AD
:1071A0000F96821793070CF451C02091440430913C
:1071B0004504C5010397281739070CF447C0C501DA
:1071C0004496821793070CF441C0EE818A81E81738
:1071D00009F03CC0E150EE0FEE0FE9298D8181509E
:1071E00090E0EE0FEE0F9C0103E0359527950A9590
:1071F000E1F7E22BF0E0E658FC4F8770907021E059
:1072000030E002C0220F331F8A95E2F78081822787
:1072100080838E010B5F1F4FC80162DBF82EF220C6
:10722000C8010E94B72F882311F0A0E8FA2AC601EE
:10723000B5014F2DCCDB88EE93E0E0E9F1E031972A
:10724000F1F70197D1F7332433944ECFCE01059651
:107250000E94892F20E230E0C20ED31E38EFC31601
:10726000D10409F092CF88E190E0A80EB91E98EE03
:10727000A916B10409F42FCD18E1C12ED12C85CF68
:107280003324832D2896DEBFCDBFCF91DF911F9190
:107290000F91FF90EF90DF90CF90BF90AF909F90B5
:1072A0008F907F906F905F904F903F902F900895B8
:1072B000F894AAC3FC0105900020E9F78095909509
:1072C0008E0F9F1F0895AEE0B0E0E8E6F9E337C304
:1072D0000D891E898EE08C831A8309838FEF9FE7C7
:1072E0009E838D839E01275E3F4FCE0101966F895D
:1072F000788DA90109D02F813885020F131FF8015D
:1073000010822E96E4E037C3ABE0B0E0E9E8F9E3A1
:1073100008C33C012B015A01FC01178216828381AC
:1073200081FD03C06FEF7FEFB9C19AE0892E1E0186
:107330000894211C311CF3012381F20123FD859166
:1073400023FF81912F01882309F4A5C1853239F4E7
:1073500023FD859123FF81912F01853221F490E057
:10736000B301EFD1E8CF982FFF24EE249924FFE159
:10737000FF15D0F09B3269F09C3228F4903259F01E
:10738000933291F40EC09D3249F0903369F441E09C
:1073900024C052E0F52A84E0F82A28C098E0F92AAF
:1073A00025C0E0E1FE2A22C0F7FC29C0892F8053C6
:1073B0008A3070F4F6FE05C0989C902C1124980E2B
:1073C00015C0E89CE02C1124E80EF0E2FF2A0EC064
:1073D0009E3229F4F6FC5FC140E4F42A07C09C36D3
:1073E00019F450E8F52A02C0983649F4F20123FD59
:1073F000959123FF91912F01992309F0B8CF892FFF
:107400008554833018F08052833038F444E050E0E3
:10741000A40EB51E5FE359830FC0933631F0933746
:1074200079F0933509F052C01FC0F501808189833E
:1074300042E050E0A40EB51E610101E010E011C071
:10744000F501C080D180F6FC03C06FEF7FEF02C072
:10745000692D70E042E050E0A40EB51EC60166D171
:107460008C015FE7F52213C0F501C080D180F6FCE6
:1074700003C06FEF7FEF02C0692D70E042E050E083
:10748000A40EB51EC60147D18C0150E8F52AF3FEC3
:1074900006C018C080E290E0B30153D1EA948E2D6B
:1074A00090E008171907B0F30DC0F601F7FC8591BD
:1074B000F7FE81916F0190E0B30143D1E110EA94AE
:1074C000015010400115110581F7E2C0943611F00A
:1074D000993661F5F7FE08C0F501208131814281BE
:1074E000538184E090E00AC0F501808191819C0184
:1074F000442737FD4095542F82E090E0A80EB91E36
:107500009FE6F92257FF09C0509540953095219587
:107510003F4F4F4F5F4FE0E8FE2ACA01B901A1017A
:107520002AE030E03AD1D82ED2183FC0953729F45E
:107530001F2D1F7E2AE030E01DC01F2D197F9F36B2
:1075400061F0903720F4983509F0A5C00FC090374E
:1075500039F0983709F09FC004C028E030E00AC035
:10756000106114FD146020E130E004C014FD1660C9
:1075700020E132E017FF08C0F5016081718182814E
:10758000938144E050E008C0F50180819181BC0105
:1075900080E090E042E050E0A40EB51EA101FDD0D5
:1075A000D82ED2188FE7F82EF122F6FE0BC05EEF30
:1075B000F522D91438F4F4FE07C0F2FC05C08FEEB2
:1075C000F82202C01D2D01C0192DF4FE0DC0FE01D0
:1075D000ED0DF11D8081803319F499EEF92208C078
:1075E0001F5FF2FE05C003C08F2D867809F01F5F74
:1075F0000F2DF3FC13C0F0FE0EC01E1510F09D2CD5
:107600000AC09D2C9E0C911A1E2D05C080E290E0B0
:10761000B30197D01F5F1E15C8F304C01E1510F4E8
:10762000E11A01C0EE2404FF0EC080E390E0B30134
:1076300088D002FF1BC001FD03C088E790E00EC0A8
:1076400088E590E00BC0802F867881F001FF02C0B2
:107650008BE201C080E2F7FC8DE290E0B30171D0D3
:1076600005C080E390E0B3016CD09A94D914C8F3BC
:10767000DA94F101ED0DF11D808190E0B30161D04C
:10768000DD20B1F705C080E290E0B3015AD0EA9462
:10769000EE20C9F750CEF30166817781CB012B969E
:1076A000E2E15BC1DC01CB01FC01F999FECF06C030
:1076B000F2BDE1BDF89A319600B40D9241505040B0
:1076C000B8F70895F999FECF92BD81BDF89A992730
:1076D00080B50895DC01A40FB51F4150504040F023
:1076E000CB01840F951F2E9105D041505040D8F703
:1076F0000895262FF999FECF92BD81BDF89A019782
:1077000000B4021639F01FBA20BD0FB6F894FA9AE9
:10771000F99A0FBE0895FC01059061507040011068
:10772000D8F7809590958E0F9F1F0895FC016150AA
:10773000704001900110D8F7809590958E0F9F1F93
:1077400008950F931F93CF93DF938C01EB018B81EF
:1077500081FF1BC082FF0DC02E813F818C819D81E6
:107760002817390764F4E881F9810193F983E883E4
:1077700006C0E885F985802F0995892B31F48E8123
:107780009F8101969F838E8302C00FEF1FEFC80178
:10779000DF91CF911F910F910895FA01AA27283008
:1077A00051F1203181F1E8946F936E7F6E5F7F4FCE
:1077B0008F4F9F4FAF4FB1E03ED0B4E03CD0670F4A
:1077C000781F891F9A1FA11D680F791F8A1F911D9D
:1077D000A11D6A0F711D811D911DA11D20D009F4ED
:1077E00068943F912AE0269F11243019305D31932F
:1077F000DEF6CF010895462F4770405D4193B3E018
:107800000FD0C9F7F6CF462F4F70405D4A3318F0BE
:10781000495D31FD4052419302D0A9F7EACFB4E06F
:10782000A6959795879577956795BA95C9F7009727
:107830006105710508959B01AC010A2E06945795C8
:10784000479537952795BA95C9F7620F731F841F1F
:10785000951FA01D0895629FD001739FF001829F24
:10786000E00DF11D649FE00DF11D929FF00D839FCF
:10787000F00D749FF00D659FF00D9927729FB00D6C
:10788000E11DF91F639FB00DE11DF91FBD01CF017F
:1078900011240895991B79E004C0991F961708F0E8
:1078A000961B881F7A95C9F78095089587FB082E47
:1078B000062687FD819567FD6195ECDF0EF49195B5
:1078C00007FC8195089597FB092E07260AD077FDBE
:1078D00004D05ED006D000201AF4709561957F4FD9
:1078E0000895F6F7909581959F4F089597FB092E7F
:1078F00005260ED057FD04D05FD00AD0001C38F406
:1079000050954095309521953F4F4F4F5F4F0895CB
:10791000F6F790958095709561957F4F8F4F9F4FAB
:1079200008952F923F924F925F926F927F928F9223
:107930009F92AF92BF92CF92DF92EF92FF920F93FE
:107940001F93CF93DF93CDB7DEB7CA1BDB0B0FB608
:10795000F894DEBF0FBECDBF09942A8839884888C5
:107960005F846E847D848C849B84AA84B984C8845B
:10797000DF80EE80FD800C811B81AA81B981CE0F52
:10798000D11D0FB6F894DEBF0FBECDBFED01089537
:10799000AA1BBB1B51E107C0AA1FBB1FA617B70735
:1079A00010F0A61BB70B881F991F5A95A9F7809551
:1079B0009095BC01CD010895A1E21A2EAA1BBB1B14
:1079C000FD010DC0AA1FBB1FEE1FFF1FA217B307AB
:1079D000E407F50720F0A21BB30BE40BF50B661FC1
:1079E000771F881F991F1A9469F760957095809585
:1079F00090959B01AC01BD01CF010895EE0FFF1FD3
:0C7A00000590F491E02D0994F894FFCF5C
:107A0C00E28093002B004F4B004162627265636809
:107A1C00656E00000000000000143C003E007A750A
:107A2C0072C3BC636B00C3846E6465726E005A755E
:107A3C0072C3BC636B0053706569636865726E00DA
:107A4C0000010202030303030404040404040404F9
:107A5C0005050505050505050505050505050505CA
:107A6C0006060606060606060606060606060606AA
:107A7C00060606060606060606060606060606069A
:107A8C00070707070707070707070707070707077A
:107A9C00070707070707070707070707070707076A
:107AAC00070707070707070707070707070707075A
:107ABC00070707070707070707070707070707074A
:107ACC00080808080808080808080808080808082A
:107ADC00080808080808080808080808080808081A
:107AEC00080808080808080808080808080808080A
:107AFC0008080808080808080808080808080808FA
:107B0C0008080808080808080808080808080808E9
:107B1C0008080808080808080808080808080808D9
:107B2C0008080808080808080808080808080808C9
:107B3C0008080808080808080808080808080808B9
:107B4C000001010201020203010202030203030409
:107B5C0001020203020303040203030403040405E9
:107B6C0001020203020303040203030403040405D9
:107B7C0002030304030404050304040504050506B9
:107B8C0001020203020303040203030403040405B9
:107B9C000203030403040405030404050405050699
:107BAC000203030403040405030404050405050689
:107BBC000304040504050506040505060506060769
:107BCC000102020302030304020303040304040579
:107BDC000203030403040405030404050405050659
:107BEC000203030403040405030404050405050649
:107BFC000304040504050506040505060506060729
:107C0C000203030403040405030404050405050628
:107C1C000304040504050506040505060506060708
:107C2C0003040405040505060405050605060607F8
:107C3C0004050506050606070506060706070708D8
:00000001FF
